:100000000C94E50B0C941D0C0C941D0C0C941D0C05
:100010000C941D0C0C941D0C0C941D0C0C941D0CBC
:100020000C941D0C0C941D0C0C94FE300C94E631B9
:100030000C94BA180C941D0C0C941D0C0C941D0CF3
:100040000C941D0C0C941D0C0C941D0C0C941D0C8C
:100050000C941D0C0C94DA300C941D0C0C941D0C9B
:100060000C941D0C0C941D0C0C941D0C0C941D0C6C
:100070000C941D0C0C941D0C0C941D0C0C941D0C5C
:100080000C941D0C0C941D0C0C941D0C0C941D0C4C
:100090000C941D0C0C941D0C0C941D0C0C941D0C3C
:1000A0000C941D0C0C941D0C0C941D0C0501098066
:1000B000A101850319012AB700150126B700950192
:1000C00075108100C0050C0901A101850419012AE0
:1000D000A002150126A002950175108100C005013E
:1000E0000906A1018506050719E029E71500250184
:1000F0009508750181020507190029EF15002501F2
:1001000095F075018102050819012905950575010C
:100110009102950175039101C00660FF0961A1017B
:100120000962150026FF00952075088102096315F4
:100130000026FF00952075089102C005010906A15F
:1001400001050719E029E7150025019508750181CA
:10015000029501750881010507190029FF15002680
:10016000FF0095067508810005081901290515008D
:100170002501950575019102950175039101C00056
:10018000AF00AE07087F0807003E5B4F5B3E003EB6
:100190006B4F6B3E001C3E7C3E1C00183C7E3C18A6
:1001A000001C577D571C001C5E7F5E1C0000183C25
:1001B000180000FFE7C3E7FF00001824180000FF45
:1001C000E7DBE7FF0030483A060E002629792926AA
:1001D00000407F05050700407F05253F005A3CE7AA
:1001E0003C5A007F3E1C1C0800081C1C3E7F00146B
:1001F000227F2214005F5F005F5F0006097F017F9E
:1002000000006689956A0060606060600094A2FFEB
:10021000A2940008047E04080010207E201000082C
:10022000082A1C0800081C2A0808001E10101010BC
:10023000000C1E0C1E0C0030383E383000060E3EFE
:100240000E060000000000000000005F000000003B
:100250000700070000147F147F1400242A7F2A124D
:100260000023130864620036495620500000080736
:10027000030000001C224100000041221C00002A53
:100280001C7F1C2A0008083E08080000807030000F
:10029000000808080808000000606000002010083E
:1002A0000402003E5149453E0000427F400000727A
:1002B00049494946002141494D33001814127F1025
:1002C000002745454539003C4A4949310041211143
:1002D000090700364949493600464949291E0000A8
:1002E0000014000000004034000000000814224107
:1002F00000141414141400004122140800020159BF
:100300000906003E415D594E007C1211127C007FAF
:1003100049494936003E41414122007F4141413E29
:10032000007F49494941007F09090901003E4141D7
:100330005173007F0808087F0000417F41000020C2
:1003400040413F01007F08142241007F404040406F
:10035000007F021C027F007F0408107F003E4141A5
:10036000413E007F09090906003E4151215E007FA0
:10037000091929460026494949320003017F010332
:10038000003F4040403F001F2040201F003F4038BA
:10039000403F006314081463000304780403006101
:1003A00059494D4300007F4141410002040810209B
:1003B00000004141417F000402010204004040402E
:1003C0004040000003070800002054547840007F9C
:1003D0002844443800384444442800384444287FA2
:1003E0000038545454180000087E09020018A4A4D0
:1003F0009C78007F080404780000447D40000020C1
:1004000040403D00007F102844000000417F400034
:10041000007C04780478007C0804047800384444A4
:10042000443800FC182424180018242418FC007CEC
:10043000080404080048545454240004043F44248D
:10044000003C4040207C001C2040201C003C4030F0
:10045000403C004428102844004C9090907C00447C
:1004600064544C440000083641000000007700004E
:10047000000041360800000201020402003C26236D
:10048000263C00000000000000404040F0F8F8FF6B
:1004900038FFF8F83FF8F8FF38FFF8F8F040404030
:1004A00000000000000080C0C0C0800000C0C0800C
:1004B00000000080C0C000C0C0000080C0C00000BC
:1004C000000000C0C0C0C0C000C0C00000000000EC
:1004D000000000000000000000000000000000001C
:1004E000000000000000000000000000000000000C
:1004F00000000000000000000000000000000000FC
:100500000000C0F0F8FC3E1E06010000007F4141E3
:10051000417F007F4141417F000080C0E07E5B4F12
:100520005BFEC00000C000DCD7DEDEDED7DC00C032
:1005300000000000000000000000000000000000BB
:10054000000000000000000000494949FFFFFFFFD4
:10055000E0DFBFBF00BFBFDFE0FFFFFFFF4949494A
:1005600000000000001F3F6060E0BF1F007F7F07AA
:100570001E381E077F7F007F7F0E1F3B71600000CB
:100580000000007F7F0C0C0C007E7E007F7E03034A
:10059000007F7E03037E7E03037F7E000F3E703C60
:1005A000063C703E0F00327B49493F7E007F7E0350
:1005B00003001E3F69696F26000000000000000074
:1005C0000000030F1F3F3C7870600000007F414136
:1005D000417F007F4141417F00307B7F7830202088
:1005E00030787F3B0003000F7F0F0F0F7F0F00035A
:1005F00000000000000000000000000000000000FB
:10060000000000000000000000010101070F0F7F43
:100610000F7F0F0F7E0F0F7F0F7F0F0F070101015D
:1006200000000000000000000000010100000000C8
:1006300000000000000000000000000000000000BA
:1006400000000000000000000000000000000000AA
:10065000000000000000000000000000000000009A
:10066000000000000000000000000000000000008A
:10067000000000000000000000000000000000007A
:10068000000000000000000000000000000000006A
:10069000000000000000000000000000000000005A
:1006A000000000000000000000000000000000004A
:1006B000000000000000000000000000000000003A
:1006C000000000000000000000000000000000002A
:1006D000000000000000000000000000000000001A
:1006E000000000000000007E0F00D4FFFFFFC700E5
:1006F00000007800000000000000002A2B28000005
:1007000000000000000000000000000000002900C0
:100710000000002C1E3420212224342627252E36CA
:100720002D3738271E1F2021222324252633333638
:100730002E37381F0405060708090A0B0C0D0E0F8B
:10074000101112131415161718191A1B1C1D2F310E
:1007500030232D350405060708090A0B0C0D0E0F72
:10076000101112131415161718191A1B1C1D2F31EE
:1007700030354C09025B00030100A0FA09040000B7
:1007800001030101000921110100012244000705B4
:10079000810308000109040100020300000009218F
:1007A0001101000122220007058203200001070534
:1007B00003032000010904020001030000000921D5
:1007C00011010001226D00070584032000011201C0
:1007D0000002000000082837492901000102030136
:1007E0001C037600690061006C003A006600360068
:1007F0003400630032006200330063000000120323
:1008000042006F006E0067006F00500061006400DE
:1008100000000C034C006C0033006D006100000010
:1008200004030904A800000000002400250026009D
:100830002100220023001E001F0020002C000000C9
:1008400000002C002C002C002C002C002C002C0074
:100850002C002C002C00000000002C002C002C0090
:100860002C002C002C002C002C002C002C00000054
:1008700000002C002C002C002C002C002C002C0044
:100880002C002C00AA00A9000100010001000100B9
:100890000100010000DA0281FFD9F1DB20A4A62EBD
:1008A000AF00A0C0D30000A1C8D30000AED580A87F
:1008B0001F408D142000FD377A585A000004E6D6F8
:1008C000B4460200210116000000742FE5A3E001E8
:1008D0000500AA5D003D8889C65436C3174FE4D48D
:1008E000201442FD004CB881A1EBC560983D640323
:1008F0002DCF41150E53BAB80C7A103502F4C7C08B
:10090000873C401FDCEE8A78829BF11297EC019BBA
:100910009ABDA8977AF42257C3B1E60C2CBDDFCE5E
:10092000DA86942738B17A8A00BC90A1EC02492675
:10093000129725BC2BA94B02941E770744CEB80C06
:10094000B6D4F57E983CE549072963D940BB9D4064
:10095000ECD1255D523A39A74061166A2C8B16CD31
:10096000E7F63D56B511AF46F61421E5DD53871D78
:10097000D61D5CF08819E990B801AE135C7B0000CD
:100980000000ADFC63A576B264F30001C6018602E7
:1009900000004D3D32F2B1C467FB020000000004CC
:1009A000595A504F52514A4D4B4E2A4C2F30B6B7E0
:1009B000ABACBBBCA9AABDBE0D0E0B0F1A0508053A
:1009C0000905071811130408120C000000000000AC
:1009D0000000000000000000000000000000000017
:1009E0000000000000000000000000000000000007
:1009F00000000000000000000000000000808000F7
:100A0000000000008040402020202010101010081E
:100A100004020101020C30408000000000000000D0
:100A2000F8F8F8F8000000000080800000000000E6
:100A300000000000000000000000000000000000B6
:100A40000000000000000080808000000000000026
:100A50000000000000000000000000000000000096
:100A60000000000000000000000000000000000086
:100A700000000000000000000000001EE100000176
:100A800001020281808000008080000000000000E0
:100A90000000008000303000000101020408102036
:100AA0004387070100B8BCBE9F5F5F4F4C202020EA
:100AB00020101010100808080808C404C404C40258
:100AC000C202C2010101010000000000000000009C
:100AD0000000000000000000000000000000000016
:100AE0000000000000000000000000000000000006
:100AF0000000000000000000000080700C030000F7
:100B0000180605989984437C4141404020212212D7
:100B10001111110908080808040408081010101021
:100B200010110F013D7CFCFCFCFCFC3C0C000000A7
:100B300000000000000000AAAAFFFFC3BF7F037FE0
:100B4000BFC3FFFFAAAA00000000000000000000D1
:100B50000000000000000000000000000000008015
:100B6000808080404040402020202010101010083D
:100B70000808080804040404040203020201010135
:100B80000101010000000000000000000000000062
:100B90000000000000000000000000000000000055
:100BA000000000000000000103030000000000003E
:100BB000000000000000000202071F071F071C07BB
:100BC0001F071F07020200000000000000000000D5
:100BD0000000000000000000000000000000000015
:100BE0000000000000000000000000000000000005
:100BF00000000000000000000000000000808000F5
:100C0000000000008040402020202010101010081C
:100C100004020101020C30408000000000000000CE
:100C200000000000000000000000000000000000C4
:100C300000000000000000000000000000000000B4
:100C40000000000000000080808000000000000024
:100C50000000000000000000000000000000000094
:100C60000000000000000000000000000000000084
:100C700000000000000000000000001EE100000174
:100C8000010202010000000080800000000000005E
:100C900000000080003030000001E11A0609313503
:100CA000018A7C00008080808040404040202020DD
:100CB00020101010100808080808C404C404C40256
:100CC000C202C2010101010000000000000000009A
:100CD0000000000000000000000000000000000014
:100CE0000000000000000000000000000000000004
:100CF0000000000000000000000080700C030000F5
:100D0000000000000000000001010040A0212212AC
:100D1000111111090808080804040404040402025B
:100D200002010101010000000000000000000000BD
:100D300000000000000000AAAAFFFFC3BF7F037FDE
:100D4000BFC3FFFFAAAA00000000000000000000CF
:100D50000000000000000000000000000000008013
:100D6000808080404040402020202010101010083B
:100D700008080808040404040402037A7A797979DB
:100D80007939310202040408080808080700000045
:100D9000303C7C7C7E7E7E7E0000000000000000F7
:100DA0000000000000000000000000000000000043
:100DB000000000000000000202071F071F071C07B9
:100DC0001F071F07020200000000000000000000D3
:100DD0000000000000000000000000000000000013
:100DE0000000000000000000000000000000000003
:100DF00000000000000000000000000000000000F3
:100E00000000000080404020202020101010101012
:100E100008080404040830408000000000000000BE
:100E200000000000000000000000000000000000C2
:100E300000000000000000000000000000000000B2
:100E40000000000000000080808000000000000022
:100E50000000000000000000000000000000000092
:100E60000000000000000000000000000000000082
:100E70000000000000000000000000186482020270
:100E8000020202010000000080800000000000005B
:100E90000000008000303000C0C1C1C20408102032
:100EA0004080000000808080804040404020202022
:100EB00020101010100808080808C404C404C40254
:100EC000C202C20101010100000000000000000098
:100ED0000000000000000000000000000000000012
:100EE0000000000000000000000000000000000002
:100EF00000000000000000000000C03804030000F3
:100F000000000000000C0C0C0D010040A02122127A
:100F1000111111090808080804040808101010101D
:100F200010110F010100000000000000000000008F
:100F300000000000000000AAAAFFFFC3BF7F037FDC
:100F4000BFC3FFFFAAAA00000000000000000000CD
:100F50000000000000000000000000000000008011
:100F60008080804040404020202020101010100839
:100F70000808080804040404040203020201010131
:100F80000101010202040408080808080700000023
:100F90000000000000000000000000000000000051
:100FA0000000000000000000000000000000000041
:100FB000000000000000000202071F071F071C07B7
:100FC0001F071F07020200000000000000000000D1
:100FD0000000000000000000000000000000000011
:100FE0000000000000000000000000000000000001
:100FF00000000000000000000000000000000000F1
:101000000000000080404020202020101010101010
:1010100008080404040830408000000000000000BC
:1010200000000000000000000000000000000000C0
:1010300000000000000000000000000000000000B0
:101040000000000000000080808000000000000020
:101050000000000000000000000000000000000090
:101060000000000000000000000000000000000080
:10107000000000000000000000000018648202026E
:101080000202020100000000808000000000000059
:101090000000008000303000C0C1C1C20408102030
:1010A0004080000000808080804040404020202020
:1010B00020101010100808080808C404C404C40252
:1010C000C202C20101010100000000000000000096
:1010D0000000000000000000000000000000000010
:1010E0000000000000000000000000000000000000
:1010F00000000000000000000000C03804030000F1
:1011000000000000000C0C0C0D010040A021221278
:10111000111111090808080804040808101010101B
:1011200010110F010100000000000000000000008D
:1011300000000000000000AAAAFFFFC3BF7F037FDA
:10114000BFC3FFFFAAAA00000000000000000000CB
:10115000000000000000000000000000000000800F
:101160008080804040404020202020101010100837
:10117000080808080404040404020302020101012F
:101180000101010202040408080808080700000021
:10119000000000000000000000000000000000004F
:1011A000000000000000000000000000000000003F
:1011B000000000000000000202071F071F071C07B5
:1011C0001F071F07020200000000000000000000CF
:1011D000000000000000000000000000000000000F
:1011E00000000000000000000000000000000000FF
:1011F00000000000000000000000000000000000EF
:10120000000000000080804040404020202020104E
:1012100008040202041860800000000000000000C2
:1012200000000000000000000000000000000000BE
:1012300000000000000000000000000000000000AE
:10124000000000000000008080800000000000001E
:10125000000000000000000000000000000000008E
:10126000000000000000000000000000000000007E
:1012700000000000000000000000003CC20101026C
:101280000204040201000000000000000000000051
:10129000000000000060600081828284081020400D
:1012A000800000000080808080404040402020205E
:1012B00020101010100808080808C404C404C40250
:1012C000C202C20101010100000000000000000094
:1012D000000000000000000000000000000000000E
:1012E00000000000000000000000000000000000FE
:1012F00000000000000000000000807019060000DF
:1013000000000000001818181B030040A02224143D
:101310001212120B08080808050509091010101010
:1013200010110F010100000000000000000000008B
:1013300000000000000000AAAAFFFFC3BF7F037FD8
:10134000BFC3FFFFAAAA00000000000000000000C9
:10135000000000000000000000000000000000800D
:101360008080804040404020202020101010100835
:10137000080808080404040404020302020101012D
:10138000010101020204040808080808070000001F
:10139000000000000000000000000000000000004D
:1013A000000000000000000000000000000000003D
:1013B000000000000000000202071F071F071C07B3
:1013C0001F071F07020200000000000000000000CD
:1013D000000000000000000000000000000000000D
:1013E00000000000000000000000000000000000FD
:1013F00000000000000000000000000000808000ED
:101400000000000080404020202020101010100814
:1014100004020101020C30408000000000000000C6
:1014200000000000000000000000000000000000BC
:1014300000000000000000000000000000000000AC
:10144000000000000000008080800000000000001C
:10145000000000000000000000000000000000008C
:10146000000000000000000000000000000000007C
:1014700000000000000000000000001EE10000016C
:101480000102020100000000808000000000000056
:101490000000008000303000C0C1C1C2040810202C
:1014A000408000000080808080404040402020201C
:1014B00020101010100808080808C404C404C4024E
:1014C000C202C20101010100000000000000000092
:1014D000000000000000000000000000000000000C
:1014E00000000000000000000000000000000000FC
:1014F0000000000000000000000080700C030000ED
:1015000000000000000C0C0C0D010040A021221274
:101510001111110908080808040408081010101017
:1015200010110F0101000000000000000000000089
:1015300000000000000000AAAAFFFFC3BF7F037FD6
:10154000BFC3FFFFAAAA00000000000000000000C7
:10155000000000000000000000000000000000800B
:101560008080804040404020202020101010100833
:10157000080808080404040404020302020101012B
:10158000010101020204040808080808070000001D
:10159000000000000000000000000000000000004B
:1015A000000000000000000000000000000000003B
:1015B000000000000000000202071F071F071C07B1
:1015C0001F071F07020200000000000000000000CB
:1015D000000000000000000000000000000000000B
:1015E00000000000000000000000000000000000FB
:1015F00000000000000000000000000000000000EB
:101600000000000080404020202020101010100812
:1016100008040202020438408000000000000000BC
:1016200000000000000000000000000000000000BA
:1016300000000000000000000000000000000000AA
:10164000000000000000008080800000000000001A
:10165000000000000000000000000000000000008A
:10166000000000000000000000000000000000007A
:1016700000000000000000000000001CE201010268
:101680000202020100000000808000000000000053
:101690000000008000303000C0C1C1C2040810202A
:1016A000408000000080808080404040402020201A
:1016B00020101010100808080808C404C404C4024C
:1016C000C202C20101010100000000000000000090
:1016D000000000000000000000000000000000000A
:1016E00000000000000000000000000000000000FA
:1016F0000000000000000000000080700C030000EB
:1017000000000000000C0C0C0D010040A021221272
:101710001111110908080808040408081010101015
:1017200010110F0101000000000000000000000087
:1017300000000000000000AAAAFFFFC3BF7F037FD4
:10174000BFC3FFFFAAAA00000000000000000000C5
:101750000000000000000000000000000000008009
:101760008080804040404020202020101010100831
:101770000808080804040404040203020201010129
:10178000010101020204040808080808070000001B
:101790000000000000000000000000000000000049
:1017A0000000000000000000000000000000000039
:1017B000000000000000000202071F071F071C07AF
:1017C0001F071F0702020000000011241FBECFEFF9
:1017D000DAE0DEBFCDBF04B603FE18C080919A05E3
:1017E00090919B05A0919C05B0919D058730904BF1
:1017F000A740B04B59F410929A0510929B05109295
:101800009C0510929D05E0E0F8E3099511E0A0E049
:10181000B1E0E6EAFAE602C005900D92AC3BB107F2
:10182000D9F725E0ACEBB1E001C01D92AA39B207AF
:10183000E1F70E943C290C94FD340C9400009C01BB
:10184000FB019A9581159F4120F5832F8170B32F5D
:10185000B270AA27732F74706627532F58704427CD
:1018600034FF0DC08295807FAB2B09F08062672B1F
:1018700009F08064452B09F0806809950895AB2B29
:1018800009F08260672B09F08460452BB1F3886012
:10189000F4CF80E0F2CF0C9449340895982F9295BC
:1018A0009F7024E0911102C020E0982F892F869527
:1018B0008695811511F02E5F982F892F8695820FBE
:1018C000089580938F05089580939005089521E0F1
:1018D00030E001C0220F8A95EAF780919005822BB3
:1018E000F3CF21E030E0A90102C0440F551F8A95D3
:1018F000E2F7CA018095909190058923E5CF9B017D
:10190000677091E001C0990F6A95EAF763E0369538
:1019100027956A95E1F7B901660F771F260F371FE4
:10192000FA01E20FF31F40E050E0682F70E0819170
:10193000DF019B01042E02C0369527950A94E2F739
:10194000217021952827292328272E934F5F5F4F49
:101950004330510561F708959C01A82FA77083E0DB
:10196000369527958A95E1F7C901880F991F820F4F
:10197000931FFB01E80FF91F40E050E080E0219148
:1019800030E00A2E02C0369527950A94E2F72170BE
:101990003327042E01C0220F0A94EAF7822B4F5FEF
:1019A0005F4F4330510559F70895482F862F903FD8
:1019B00081F0943078F4433060F4292F30E0B9019D
:1019C000660F771F620F731F640F711D42EA54E0A8
:1019D00096CF08959C5F9230E0F7642F70E04FE956
:1019E00054E0F6CF482F903FB9F0943070F4833034
:1019F00098F4292F30E0C901880F991F820F931F97
:101A000062EA74E0840F911DA7CF9C5F923020F4AE
:101A10006FE974E090E0F8CF80E008959091900530
:101A200021E030E0F90101C0EE0F8A95EAF7D90113
:101A300002C0AA0FBB1F6A95E2F7EA2B01C0220F72
:101A40004A95EAF7892F8E23E81303C0892F822B4A
:101A50003BCF2095822F8923FBCF982F90958091A3
:101A60008E05892380938E050895809186058115C2
:101A700031F0109286051092960510929505089502
:101A8000803E9105D9F1C8F48133910509F482C0F3
:101A900048F48932910509F472C08A32910509F43B
:101AA00080C0089589339105E9F082389105D1F01D
:101AB0008533910509F45EC00895843E9105D9F1FE
:101AC00048F4823E910539F1833E910549F181EE5A
:101AD00090E00895863E9105C9F1873E910509F48D
:101AE0003EC00895209197052370211164C0209174
:101AF000980523FF14C089E290E00895209197058E
:101B000020FD45C03091980530FF09C024FD24C058
:101B100083EE90E008952091970522FDF7CF089578
:101B20002091970522FD44C03091980530FD43C0B7
:101B300024FFF5CF11C02091980521FFF0CF8091AF
:101B4000970584FD09C087EE90E0089520919705E0
:101B500023FFE5CF24FFF7CF80E090E008952091A8
:101B6000970523FD2BC03091980531FFE1CF84EE1E
:101B700090E008952091970525FFD1CFBCCF20910B
:101B8000970525FD1EC02091980523FFC8CF89E346
:101B900090E008952091970526FFC1CF8AE290E05A
:101BA00008952091970526FFBACF81E390E008952C
:101BB00082EE90E0089580EE90E0089586EE90E049
:101BC000089585E390E008959091970592FF10C0E5
:101BD00041E0282F2471243009F040E031E0282F23
:101BE0002871283009F030E0431711F02CE08227EB
:101BF00093FF10C041E0282F2471243109F040E008
:101C000031E0282F2871283109F030E0431711F016
:101C10002CE082273091980530FF10C051E0282F2A
:101C20002171213009F050E041E0282F287128303F
:101C300009F040E0541711F029E0822731FF10C06D
:101C400041E0282F2171213109F040E031E0282FB7
:101C50002871283109F030E0431711F029E082277C
:101C600094FD877E08951F93CF93DF9309DFEC01E6
:101C7000811522E5920708F043C0811540E59407DD
:101C800008F0D1C0803E910530F58D3C910508F0FB
:101C9000A5C0883A910580F4853A910508F09BC06B
:101CA0008130910509F452C00497813A910508F4F6
:101CB0004DC0C0E0D0E04AC0885A91094B97C8F7A0
:101CC000C85AD0E0CC0FDD1FC05BDE4F0990D88131
:101CD000C02DD4643BC0811550E2950708F0B9C00F
:101CE000883E910598F19A9581159F4110F78D2FA7
:101CF0006BDF182FCE019927C3DEEC01D12B26C054
:101D0000C03882E5D807E8F5C03692E5D90708F073
:101D10006EC0C03422E5D207F0F4C03242E5D407E9
:101D200008F05EC08C2F8695869550E2859FC00195
:101D30001124C37021E030E0A90102C0440F551FF7
:101D4000CA95E2F7EA01C82BD92BDD68CE01DF91F5
:101D5000CF911F9108958C2F86958695877050E2BC
:101D6000859FC0011124C37021E030E0A90102C0A9
:101D7000440F551FCA95E2F7EA01C82BD92BDC683E
:101D8000E5CFC03C52E5D50768F48C2F8F71C03A7F
:101D9000D24508F042C090E0982F8827EC01C46F2C
:101DA000D06AD4CFCE01805C9245809708F081CF75
:101DB000CE0123E0880F991F2A95E1F7807E9927AD
:101DC000C370DD2721E030E0A90102C0440F551F98
:101DD000CA95E2F71DC0A497D064B8CFD065B6CF3E
:101DE000CF71D0E0DC2FCC27C16FD06AAFCF8C2F62
:101DF00086958695877020E2829FC0011124C3706A
:101E000021E030E0A90102C0440F551FCA95E2F756
:101E1000EA01C82BD92BDA6899CFD6DEC82FD0E0DB
:101E2000DC2FCC2793CF8F71CFDE93E0CC0FDD1F5B
:101E30009A95E1F7CC27DF70282F30E084FF05C0AA
:101E400090E1899F900111243327C22BD32BD069B5
:101E50007DCF992715DEEC0179CF80E00895F894C5
:101E6000E82FE295EF70F0E041A18F7021E030E0C3
:101E7000B90102C0660F771F8A95E2F7CB01962F52
:101E80009095942391A392A1892B82A3789408958D
:101E900081152CE7920741F420916C0430916D0478
:101EA000232B11F480E090E00895E6E4F5E080E073
:101EB00090E063EA77E246EC57E228E338E2778382
:101EC0006683518740873387228797878687019665
:101ED00070968430910599F70895FB01811520E2F1
:101EE000920728F4811541E0940738F408959C0185
:101EF00030522115304348F00895392F94FF02C025
:101F00003295307F2081232B208399270895462BFB
:101F100022FF0FC0982F92959F708F70892B962F5C
:101F200092959F706F70692B942F92959F704F7050
:101F3000492B982F9623961309C050E04095509551
:101F400090E04823592381E0452B09F080E0089573
:101F500023E3611101C021E334B12F7081E090E0EF
:101F600001C0880F2A95EAF7982F9095932394B98A
:101F700095B1892B85B9089523E3611101C021E34F
:101F800083B190E02F7002C0959587952A95E2F76E
:101F9000817008950F931F93CF9301E010E0082EF6
:101FA00001C0000F0A94EAF7C0918D059C2F902381
:101FB000911115C0909192059695969596958913D5
:101FC00006C01092920510929405109293057FDC42
:101FD000C027C0938D05CF911F910F91089581DC8B
:101FE000F7CF90912E0589029001112437FF03C08D
:101FF00080932E0508952F3731051CF4980F909388
:102000002E0508959C0180E090E0F901E80FF91F8A
:10201000E491E41307C091E08927F901E80FF11D6D
:10202000849108950196861780F380E00895FA015F
:10203000309709F009950895E0919504F091960480
:10204000309739F00190F081E02D309711F009952B
:10205000089580E00895A3E0B0E0E1E3F0E10C949E
:10206000BF339C0180910A0290910B028217930763
:10207000B1F030930B0220930A02E0919504F091A5
:102080009604309761F00084F185E02D309739F0A7
:1020900083E089833B832A83CE01019609952396A9
:1020A000E2E00C94DB33A3E0B0E0E9E5F0E10C946E
:1020B000BF339C0180910802909109028217930717
:1020C000B1F03093090220930802E0919504F09159
:1020D0009604309761F00084F185E02D309739F057
:1020E00084E089833B832A83CE0101960995239658
:1020F000E2E00C94DB3390911701913091F0A0EC69
:10210000B1E0EFEF90E02D91821751F0EF3F19F41D
:10211000211101C0E92F9F5F9630A9F7EF3FC9F465
:1021200008959091970597FFEACFE82FE695E695F9
:10213000E695803FA8F7F0E0EA53FE4F877021E074
:1021400030E001C0220F8A95EAF78281822B8283D8
:1021500008950E2E000CFF0BE254FE4FF8CF909125
:102160001701913021F49091970597FD0CC0E0EC98
:10217000F1E09191891302C0DF011E9251E0E63C2B
:10218000F507B9F70895E82FE695E695E695803FBF
:10219000C8F7F0E0EA53FE4F877021E030E0A90174
:1021A00002C0440F551F8A95E2F7CA0180959281BB
:1021B0008923828308958091160108952FB7F8949A
:1021C00060910402709105028091060290910702CD
:1021D0002FBF08950895FC019B018091FA01909111
:1021E000FB018617970740F0672B29F48091E800E0
:1021F0008E778093E800C90140E0009741F44111D7
:1022000006C08091E80082FF2FC080E008952091F1
:102210006E042115A9F12530A9F12091E80023FDD4
:102220002DC02091E80022FDECCF2091E80020FF96
:10223000E4CF3091F3002091F200009719F028309C
:10224000310558F041E02830310509F040E0209197
:10225000E8002E772093E800D0CF41914093F10021
:1022600001972F5F3F4FE9CF80916E04811541F0B8
:10227000853041F08091E80083FFC3CF81E008956D
:1022800082E0089583E008958091F40187FF13C0F0
:102290008091E80082FF06C08091E8008B778093F0
:1022A000E800089580916E048111F2CF0895809125
:1022B0006E048115D9F38091E80080FFF8CF8091FA
:1022C000E8008E77ECCF2091E4003091E50095E6B0
:1022D000A9012091EC00822F817020FF06C080911F
:1022E000E80080FF06C080E008952091E80022FD0C
:1022F0001AC080916E04811589F0853089F0809133
:10230000EB0085FD0FC02091E4003091E5004217FD
:102310005307F9F29A95E1F684E0089582E0089572
:1023200083E0089581E00895E8EDF0E080818E7FFC
:1023300080831092E2001092DA001092E100A0EE89
:10234000B0E08C9181608C9380818F77808319BC01
:10235000A7EDB0E08C918E7F8C9380818F7E8083FF
:102360001092F3010895E0919504F091960430974E
:1023700039F00284F385E02D309711F060E2099581
:10238000089590919205892F8D7F80939205292F32
:102390002570211110C091FF0EC09091980592FFF9
:1023A0000AC08695869586959CDA109292051092C1
:1023B0009405109293050895EF92FF920F931F9347
:1023C000CF93DF93A0913B02B0913C029D012D532E
:1023D0003240BD016D537040613042E0740710F02F
:1023E00060E072E04091390250913A02FC01EE2423
:1023F000E394F12C2617370748F050933A024093A4
:102400003902CDB7DEB7E6E00C94D73384919D91C5
:102410008917A1F08D0101501109E8018883C901D4
:10242000C5E096958795CA95E1F7E70102C0CC0F04
:10243000DD1F8A95E2F7CE014C2B592B2F5F3F4FC2
:102440003196D8CF2F923F92CF93DF93E1018091C5
:10245000990581111DC0E881F981818590E001967F
:1024600065E070E00E94F2338187E881F98121857F
:10247000422F50E084E090E0821B910997FF02C058
:10248000CA010497982F8827990F8653924F94DF9B
:10249000E881F981808590E0019681709927808795
:1024A000E881F9812085422F50E081E090E0821B95
:1024B000910997FF02C0CA010197982F8827990FA9
:1024C0008653964F79DFDF91CF913F902F900895FB
:1024D000982F9093E900891771F07091EC0020918A
:1024E000ED005091F00021FD09C09F5F973089F702
:1024F0008093E9000895762F242F50E03091EB006F
:102500003E7F3093EB003091ED003D7F3093ED0046
:102510003091EB0031603093EB007093EC0020932E
:10252000ED005093F0002091EE0027FDDECF0895DE
:10253000A0E0B0E0EEE9F2E10C94B933C8EDD0E0F0
:1025400088818F7E8883E7EDF0E0808181608083E1
:1025500084E082BF81E08093F30188818E7F88834D
:1025600002EE10E0F80110821092DA0081EEC82E1F
:10257000D12CF601108288818F77888388818068CA
:10258000888388818F7D888319BC10926E04109295
:10259000F201109247041092F10190EEE92EF12C15
:1025A000F70180818B7F808388818160888342E00E
:1025B00060E080E08DDFF60180818E7F8083F8010E
:1025C000808181608083808188608083F701808141
:1025D0008E7F8083888180618883CDB7DEB7E8E015
:1025E0000C94D53381E08093E00080E28093D800A2
:1025F0001092C9008FE19EE40197F1F700C000003E
:1026000087E090EBDC0180939A0590939B05A09363
:102610009C05B0939D0588E19CE00FB6F894A895C1
:10262000809360000FBE90936000FFCF0F931F93C5
:10263000CF93DF938B01EA0190916E04943051F5B2
:102640008093E9008FEF9091E80095FD06C095ED2D
:102650009A95F1F700008A95B1F78091E80085FF1F
:1026600019C031DE811111C08091E80085FD06C0DE
:102670008091E8008E778093E800F3CFF801819194
:102680008F018093F100219779F78091E8008E7790
:102690008093E800DF91CF911F910F910895792FDA
:1026A000603229F440E250E0682F82E0BFCF089505
:1026B000CF93DF93D82FC92F48E050E0682F792FB0
:1026C00081E0B4DF88E0ED2FFC2FACEFB1E00190AA
:1026D0000D928A95E1F7DF91CF910895BC0140E218
:1026E00050E084E0A3CFBC0143E050E084E09ECF03
:1026F0009091980592FB222720F9281769F080FB1A
:1027000092F990939805609197057091980584E0EF
:1027100090E00E94E23435CE08951F93CF93DF936B
:10272000962F122F632F282F292B2430C8F44330E3
:10273000B8F4C42FD0E0CC0FDD1F26E0929FC00D6F
:10274000D11D112498E1899FC00DD11D1124CE0106
:1027500089960E94C834612FCE018A960E94C8349F
:10276000DF91CF911F9108950F931F93CF93DF9324
:10277000962F142F022F632F8430E8F491111BC081
:1027800024E0829FE0011124C757DF4F81E08427B6
:102790009E01280F311D280F311DC9010E94C83428
:1027A00081E090E0111102C083E090E0602F8C0F77
:1027B0009D1F0E94C834DF91CF911F910F91089502
:1027C0000F931F93CF93DF93982F962B943020F580
:1027D000433010F5C42FD0E0CC0FDD1F26E0629F00
:1027E000C00DD11D112438E1839FC00DD11D1124CE
:1027F000CE0189960E94AC34082F10E0102F0027DC
:10280000CE018A960E94AC349801282BC901DF9131
:10281000CF911F910F91089580E090E0F8CFFF9243
:102820000F931F93CF93DF93F42E843040F5611103
:1028300026C024E0829F8001112407571F4F81E0AA
:1028400084279801280F311D280F311DC9010E94CE
:10285000AC34C82FD0E0DC2FCC2781E090E0F11021
:1028600002C083E090E0800F911F0E94AC349E0173
:10287000282BC901CDB7DEB7E5E00C94D83380E052
:1028800090E0F8CF462F672F2091710430917204A9
:10289000232BB9F4703F39F4403F99F480916F04D1
:1028A000909170040895743028F4433050F48430CB
:1028B00040F486CF7D3F41F4411103C041E08430B4
:1028C00048F080E090E008957C3FD9F74111F9CFBE
:1028D0008430B8F760E0A3CFA0E0B0E0E2E7F4E135
:1028E0000C94BA337C010091900580918F05082BE0
:1028F000C3E0D0E010E0C8010C2E02C0959587958A
:102900000A94E2F780FD09C02197A8F7D12C8D2DFC
:10291000CDB7DEB7E7E00C94D633DC2EB7018C2FB1
:10292000B1DFA1D9019781F3F2CF0F931F93CF931A
:10293000FC0186819781009781F485810081118156
:10294000811579F0611569F0C801C6DFC82F682FBD
:10295000C8012BD8B8018C2F95DFCF911F910F9113
:102960000895C8013FD8C82FF5CF382F292FCB01A4
:10297000A32FB22F8F3023E09207A105B10520F4D9
:102980008F509F4F0C94AC3480E0089585E290E026
:102990000E94AC34893189F486E290E00E94AC3424
:1029A0008B3859F487E290E00E94AC3491E08A378A
:1029B00009F090E0892F8170089580E0FCCFAAE0B3
:1029C000B0E0E5EEF4E10C94B233C0906C04D0902A
:1029D0006D0481E090E090936D0480936C0434E882
:1029E000E32E38E0F32EA12CB12C10E0350100E0ED
:1029F00014C0F40125913591452D602F812F8DDE76
:102A000022E0820E911C539433E05312F2CF83E004
:102A1000680E711C0F5F043049F0C301880F991FC5
:102A2000FC01EC5DF74F4F01512CE3CFF7012591ED
:102A3000359141E060E0812F97DEF70132962591D4
:102A4000359140E060E0812F8FDEF4E0EF0EF11C65
:102A50001F5F2CE0A20EB11C143009F0C7CF1A8200
:102A600019821C821B821E821D8218861F8288EC9E
:102A700090E09A8789874AE050E069E970E08E012A
:102A80000F5F1F4FC8010E94E6344AE050E063EA3E
:102A900070E0C8010E94E6344AE050E06DEA70E060
:102AA000C8010E94E6344AE050E067EB70E0C801DC
:102AB0000E94E63486E0F80111928A95E9F781ECEC
:102AC000E82EF12C46E050E0B701C8010E94E63440
:102AD000F6E0EF0EF11C21EFE216F10499F7D09227
:102AE0006D04C0926C042A96EFE00C94CE33A6E0FD
:102AF000B0E0EDE7F5E10C94BA3304EE14E081ECBC
:102B0000E82EF12C98E0D92E46E050E0B701CE0136
:102B100001960E949C34F8018D2D11928A95E9F757
:102B2000B8016C5F7F4F89819A81D7D9F801918371
:102B30008083B8016B5F7F4F8B819C81CED9F80178
:102B4000938382838D8186838E818783F6E0EF0E67
:102B5000F11C085F1F4F81EFE816F104A9F62696D5
:102B6000E7E00C94D633282FCB01243070F44AE0F0
:102B7000249F90011124B90167567F4F4AE050E02D
:102B80000E949C3480E090E008958FEF9FEF0895BD
:102B9000AB0124E630E0BC0188E70E9404339C01CD
:102BA00081E0232B09F080E0089580913F04811596
:102BB00061F080913E04811541F062E070E081E8AF
:102BC00091E0E6DF811110923E04089580913F0468
:102BD0008115E9F0F3DADC01CB01805A9541AF4F62
:102BE000BF4F8093400490934104A0934204B0935C
:102BF000430480913E0481110AC062E070E08FE7D7
:102C000091E0C6DF811519F081E080933E040895BC
:102C1000A0E1B0E0EEE0F6E10C94B133FE013196B4
:102C200080E1DF011D928A95E9F701E310E091EF61
:102C3000A92EB12C2FE0422E23E0522E612C712CB4
:102C40004F0173016201B1E14B165104610471043B
:102C50001CF080E1C82ED12CA601B501C4010E9450
:102C6000B934AC0CBD1C0D2C000CEE08FF084C1840
:102C70005D086E087F080150104019F76096E0E18A
:102C80000C94CD336FEF85E290E00E94C8346FEF73
:102C900086E290E00E94C8346FEF87E290E00E94E5
:102CA000C83460E088E290E00E94C83488DEB0DF7B
:102CB00069E185E290E00E94C8346BE886E290E02A
:102CC0000E94C8346AE787E290E00C94C834CF933E
:102CD000DF93682F80913B0290913C026A30B1F4FF
:102CE000209144048D539240622F70E00E949B33E8
:102CF000281B822F66E00E94E633C82FC15018F4CB
:102D0000DF91CF91089580E2E2DFF8CF6D30D9F402
:102D10009C012D53324040914404642F70E0C9015E
:102D20000E949B33481BC901840F911D811522E02D
:102D3000920710F080E090E0835C9D4F90933C02FE
:102D400080933B02DDCF26E0FC01ABEEB1E00190C9
:102D50000D922A95E1F7603E08F458C026E0FC0188
:102D600011922A95E9F7C0913B02D0913C0246E0CE
:102D700050E0BE018BEE91E00E9488349E012D53FD
:102D80003240892B41F1C90145E0969587954A95D6
:102D9000E1F741E050E0BA0102C0660F771F8A9563
:102DA000E2F7CB016091390270913A02862B972BA2
:102DB000B9016B5F7F4FE5E076956795EA95E1F79E
:102DC00002C0440F551F6A95E2F7842B952B909310
:102DD0003A02809339022A5F3F4F40914404642FA6
:102DE00070E0C9010E949B33481B463010F4240F49
:102DF000311D211572E0370710F020E030E0235C30
:102E00003D4F30933C0220933B027ACFF6E06F9F18
:102E1000B00111246D577E4F46E050E00E947F3490
:102E2000A2CFA2E1B0E0E7E1F7E10C94AF338091EB
:102E30003F04811509F478C08DE392E090933C0241
:102E400080933B02CE0186969C878B871D821E82D3
:102E50001F82188619821A821B821C821A86198682
:102E6000988B8F8785979E878D878091990581158F
:102E700009F45EC0ABDECD80DE80EF80F8849ED9A1
:102E80006C197D098E099F09693C710581059105C1
:102E900048F094D96D837E838F839887CE010D96F9
:102EA0001C01D0DA8BD969837A838B839C838DE371
:102EB00092E090933C0280933B026091990580914F
:102EC0000001861356C080911002803309F051C072
:102ED000ECE0F2E0DF010D900020E9F78D010150F8
:102EE00011097F01E016F10608F468C080913902EB
:102EF00090913A02892B09F066C080913E048115B9
:102F000099F05CD900914004109141042091420451
:102F100030914304601B710B820B930B6F3F7F4F0B
:102F20008F4F9F4708F441DE6296E2E10C94CB3369
:102F300045D961367A4E8105910510F036DEB7CF5E
:102F4000CD80DE80EF80F88439D96C197D098E0937
:102F50009F09693C71058105910508F4A8CF2ED918
:102F60006D837E838F839887FE013D961F016ADA09
:102F70009ECF6093000180E38093100270E080E0B8
:102F800090E010920F023FE0E32E32E0F32E00E0DB
:102F900010E04AE0842E912CA12CB12CA5019401C3
:102FA0000E940534605DF70162937F01B901CA0197
:102FB0000F5F1F4F0330110589F78ACFD7018D911D
:102FC0007D0185DE8FCF80913F04811509F495CF77
:102FD00080913D04811191CFF9DD2091390230912A
:102FE0003A022115310509F488CF10E041E050E0A4
:102FF000812F90E07A01012E02C0EE0CFF1C0A9492
:10300000E2F7B70162237323672B11F41F5FF0CF40
:103010002091450420FF9BC0912F990F990F990F84
:1030200037E0390F80E023E090930301809306019D
:10303000309304012093070124E630E047E050E09C
:1030400061E071E088E70E94BB32892B09F055CF1F
:10305000B0E21B9FA00111248091450480FF83C032
:10306000E1E1F2E080E2DF011D928A95E9F7E5E314
:10307000F1E0FA8BE98B01E311E089E3A82E81E00E
:10308000B82E97E0392E44244394A989BA898D91AA
:10309000BA8BA98BF80121918F01240F352F311D97
:1030A000235C3D4FE82FF0E0EF5EFD4F80E090E0C5
:1030B000632C681A742C082E01C0770C0A94EAF766
:1030C0006901812CD6019D906D019720662D6819AC
:1030D000677070E0B92D062E01C0BB0F0A94EAF7A5
:1030E0005B2E7195619571096770772701C0969481
:1030F0006A95EAF759286081562A5082839468E0DD
:103100008612E0CF019631968830910589F689893B
:103110009A89A816B90609F0B8CF04E610E020E2B3
:1031200030E041E152E060E488E70E944F33892BB0
:1031300009F0E3CEE094F0948091390290913A0244
:103140008E219F2190933A0280933902D6CE969594
:10315000879596958795282F912F9295990F907620
:103160003FE1390F61CF435C5D4F04E610E020E2A0
:1031700030E0D9CF1F921FB61F9211248F939F93D7
:10318000AF93BF9380914604811113C080910402D4
:1031900090910502A0910602B09107024196A11DEF
:1031A000B11D8093040290930502A0930602B09390
:1031B0000702BF91AF919F918F911F901FBE1F90EB
:1031C00018952FB7F8948091040290910502A09170
:1031D0000602B09107022FBF0895CF93DF93C091ED
:1031E0008E0580919105C82B80918605811501F18E
:1031F000E8DF2091950530919605821B930B883866
:10320000934110F00E94350DD091860580911701F1
:10321000813021F48091970587FD0EC086E020EC77
:1032200031E090E0815060F491110E94350DCD2B7A
:103230008C2FDF91CF9108958EE128EC31E0F1CF12
:10324000F90141919F01411569F39F5FEBCF809197
:103250001701813061F58091970587FF28C0BDDF98
:103260008093C70140E250E065E774E086EC91E0AE
:103270000E948834892BD1F080E2E6ECF1E0A5E7EA
:10328000B4E001900D928A95E1F7E0919504F091F8
:103290009604309759F00480F581E02D309731F095
:1032A00086E08093C60186EC91E00995089595DF4C
:1032B0008093BE0148E050E067E974E08EEB91E056
:1032C0000E948834892B91F388E0EEEBF1E0A7E9C6
:1032D000B4E001900D928A95E1F7E0919504F091A8
:1032E0009604309719F30280F381E02D3097F1F2C4
:1032F0008EEB91E0DACFCF93C82F8115C9F08CEF18
:103300008C0F813A90F580911701813021F48091E2
:10331000970587FD0FC0E0ECF1E08191C81701F13E
:1033200021E0E63CF207C9F78C2F0E947B108FDF6B
:10333000CF910895EC2FE695E695E695F0E0EA53F7
:10334000FE4F828190E04C2F477021E030E002C0B8
:10335000220F331F4A95E2F782239323892B21F30F
:103360008C2F0E94AF1073DFDFCF80E28C0F88308C
:1033700068F4C77081E090E001C0880FCA95EAF751
:10338000C0918E05C82BC0938E05D1CF8BE58C0FD5
:10339000833038F42C2F2452330BC9010E942B1098
:1033A000C7CFC85ACB3120F6EC2FF0E0EE0FFF1F4D
:1033B000EA57FE4F808191810E945310B9CF811549
:1033C00021F19CEF980F913A18F40E94AF103FCF73
:1033D00090E2980F983050F4877091E001C0990FF7
:1033E0008A95EAF7892F0E942D0DF1CF9BE5980F62
:1033F000933020F480E090E00C942B10885A8B31AD
:1034000020F480E090E00C94531008951F93CF9324
:10341000DF93182FEB016FDF209731F4812FCFDF7F
:10342000DF91CF911F9108958FE99FE00197F1F708
:1034300000C000002197F0CFA0E0B0E0E2E2FAE1A6
:103440000C94B833EC018881811509F1813009F0C1
:1034500045C08981813051F48A81239660E570E00E
:10346000893311F060E070E0D1DFEDCF823021F4DC
:103470008A81239640DFE7CF833021F48A81239627
:103480009EDFE1CF843041F022968111DCCFCDB7B1
:10349000DEB7E9E00C94D4338A81239620E030E053
:1034A0009AE0682F6053770BAB016A30710560F0CA
:1034B0002115310551F3EFE9FFE03197F1F700C035
:1034C000000021503109F4CF929FB001939F700DFD
:1034D00011249A01260F371F8991E3CFE82FF0E0DE
:1034E000ED50F94FB490282F26952695269530E07B
:1034F000F901ED51F94FE4908770F12C082E02C0CC
:10350000F594E7940A94E2F7E0FAEE24FF24E0F859
:10351000F901ED52F94FC490D12C082E02C0D59478
:10352000C7940A94E2F7C0FACC24DD24C0F8F9016C
:10353000ED53F94F049110E002C0159507958A9557
:10354000E2F701701127E114F10411F081EED3DEEE
:10355000C114D10411F086EECEDE60E070E08B2D58
:1035600055DFC114D10411F086EE29DFE114F10416
:1035700011F081EE24DF0115110521F060E070E00B
:103580008CE244DF21965FCF811531F090918E055A
:10359000892B80938E055BCE0895811519F00E94CA
:1035A0002D0D55CE0895811531F090919105892BFF
:1035B000809391054CCE0895811539F080959091B6
:1035C000910589238093910542CE0895809142050B
:1035D000811521F082E2F0DF1092420508951092E9
:1035E0008E05809117018130B1F48091970587FF96
:1035F00012C0E8ECF1E08EE1DF011D928A95E9F757
:1036000080E090E00E942B1080E090E00E94531038
:10361000109291051CCEE0ECF1E086E0EDCFDFDF0B
:103620002FEF84E39CE0215080409040E1F700C000
:10363000000088E19CE00FB6F894A89580936000A4
:103640000FBE90936000FFCFAAE2B0E0EAE2FBE198
:103650000C94BE3384EF91E0FC0101962091F100BF
:10366000208321E08C3F9207B9F78091F5018930E2
:1036700009F459C0C8F4823009F4B6C0833009F4A3
:1036800085C0813089F18091E80083FFEAC0809194
:10369000F4019091F5019A3008F0E3C0E92FF0E0D1
:1036A000E150FB4C0C9443348A3009F48CC08B30CD
:1036B00051F78091F401813231F78091F8019091B6
:1036C000F901892B01F78091E800877F8093E8005A
:1036D0000E94441181E09091F601911101C080E0B7
:1036E000809317017CDFCFCF8091F401813A59F6A6
:1036F0008091E800877F8093E8008091F8019091A5
:10370000F901892B61F060E080E090E070E00E94B8
:10371000EB108091E8008B778093E800B4CF68E0ED
:103720008CEF91E0F3CF8091F401813209F0ABCFBF
:103730008091F8019091F9018D7F892B09F0A3CF39
:103740008091E800877F8093E8008091E80082FF05
:1037500018C09091F3008091F200029731F48091AB
:10376000F100813011F0863021F48091F1008093D6
:1037700016018091E8008B778093E8000E94441145
:1037800082CF80916E048111E0CF7DCF8091F401D2
:10379000813A09F078CF8091F8019091F901892B55
:1037A00009F071CF8091E800877F8093E8008091D5
:1037B000E80080FFFCCF809117018093F100809199
:1037C000E8008E77D9CF8091F401813209F05BCF88
:1037D0008091E800877F8093E8000E9444118091E7
:1037E000F701809315014FCF8091F401813A09F0E0
:1037F0004ACF8091E800877F8093E8008091E800BD
:1038000080FFFCCF80911501D8CF803889F08238B5
:1038100041F58091F8018F70873018F58093E900A9
:103820008091EB0085FB882780F91092E90006C0A3
:1038300080914704880F9091F101892B9091E800C5
:10384000977F9093E8008093F1001092F1008091AF
:10385000E8008E7723C0811116C08091F601813077
:1038600011F18091E80083FF0AC08091E800877F12
:103870008093E8008091EB0080628093EB00AA9631
:10388000E3E00C94DA33823061F78091F601811520
:1038900089F01092E9008091E800877F8093E8002A
:1038A0000E944411DECF81E0933009F080E08093E4
:1038B0004704EFCF8091F8018F702FEF280F26304B
:1038C00080F68093E9002091EB0020FFE2CF933057
:1038D00031F48091EB0080628093EB00DACF90911D
:1038E000EB0090619093EB0021E030E0A90102C071
:1038F000440F551F8A95E2F74093EA001092EA00C0
:103900008091EB008860E8CF8111ABCF1091F60178
:103910001F778091E3008078812B8093E300809172
:10392000E800877F8093E8000E9444118091E800BE
:1039300080FFFCCF8091E30080688093E30083E008
:10394000111101C082E080936E048BCF80588230C9
:1039500008F087CF8091F6019091F7018C3D53E0FC
:10396000950799F583E08A838AE289834FB7F894B3
:10397000DE01139620E03EE051E2E32FF0E05093A9
:103980005700849120FF03C082958F703F5F8F7036
:103990008A30C8F0895C90E08D939D932F5F24312D
:1039A00061F74FBF8091E800877F8093E8006AE26B
:1039B00070E0CE0101960E94EB108091E8008B77B9
:1039C0008093E8004ECF805DE6CF292F3327233048
:1039D000310509F44EC078F52130310509F488C06D
:1039E0008BE590E0E3E7F7E02230310509F039CFCD
:1039F0002091E800277F2093E8002091FA01309180
:103A0000FB018217930708F49C0140E02115310562
:103A100009F073C0411171C08091E80082FDCDCFE3
:103A200080916E04811549F2853039F28091E80069
:103A300083FFF2CFC2CF8091F8019091F90121323A
:103A4000310509F446C02232310509F00ACF83302E
:103A5000910508F006CFFC01EE0FFF1FEB5DFE4F56
:103A60000190F081E02D8E5D9E4FDC018C9190E005
:103A700010C09C013327823021F12330310568F4D6
:103A8000232BB9F4E0E2F8E0E4918E2F90E0E0E23D
:103A9000F8E0009709F4E5CEABCF2330310509F00B
:103AA000E0CEE0EEF7E0E4918E2F90E0E0EEF7E07C
:103AB000F0CFE2E1F8E0E4918E2F90E0E2E1F8E06F
:103AC000E8CFEEEFF7E0E4918E2F90E0EEEFF7E035
:103AD000E0CF8330910508F0C4CEFC01EE0FFF1F4C
:103AE000E55DFE4F0190F081E02D89E090E080CF10
:103AF00082E190E0EEECF7E07BCF80916E048115DF
:103B000009F45BCF853009F458CF8091E80083FD3C
:103B100054CF8091E80082FD7FCF8091E80080FF44
:103B200075CF9091F3008091F2002115310519F0C5
:103B30008830910550F041E0089709F040E080910D
:103B4000E8008E778093E80061CF44914093F100C4
:103B50003196215031090196E8CF803809F081CEA5
:103B60008091E800877F8093E8008091F201809344
:103B7000F1006DCE811175CE1091F601123008F072
:103B800070CE8091E800877F8093E8001093F20167
:103B90000E9444111115F9F084E080936E0442E014
:103BA00061EC81E00E94681242E261EC84E00E94D4
:103BB000681242E261EC82E00E94681242E260EC2C
:103BC00083E00E94681280916E04843051F482E098
:103BD0008093180146CE8091E30087FDDDCF81E020
:103BE000DCCF81E0F5CFCF93DF93EC014A855B8595
:103BF0006E857F850E9417109B819095809191051D
:103C00008923809391058C810E942D0D20DB86E015
:103C1000FE0111928A95E9F7DF91CF910895CF9334
:103C2000DF93EC018D8181FD16C082608D838091D0
:103C300091059B81892B8093910580918E059C81B4
:103C4000892B80938E0503DB488559856E857F859A
:103C5000CE010E94171010928805109287058D8161
:103C600080FD02C0CE01BFDFDF91CF910895CF93D9
:103C7000DF93EC01A6DA8C1B9D0BDF91CF910895A9
:103C8000EF92FF920F931F93CF93DF93C62FD42F02
:103C9000122F811599F060938B0593DA9093EA01C6
:103CA0008093E901C77081E001C0880FCA95EAF7E7
:103CB0006BDCCDB7DEB7E6E00C94D73380918B0593
:103CC00068132FC0E090E901F090EA017ADA8E19CA
:103CD0009F09883C910528F500E20D0FCD1799F05A
:103CE000C770FF24F3948F2D01C0880FCA95EAF79F
:103CF00054DC083040F48D2F877001C0FF0C8A958A
:103D0000EAF78F2D41DC60E070E0812F7FDB083027
:103D100080F6D77081E001C0880FDA95EAF73DDCC4
:103D2000C8CFC77081E001C0880FCA95EAF7F7CF06
:103D3000A9E0B0E0EEE9FEE10C94AF338C01DC01C8
:103D400014968C91811509F451C161E0C8010E945B
:103D500095147C01F8018581811529F180918705F1
:103D6000909188050097F9F0E816F906E1F0FC015A
:103D7000FF278C7F9927892B09F072C024E0EE0F72
:103D8000FF1F2A95E1F7EA5BFA4F858184608583FE
:103D9000F182E082CF0143DF1092910561E0C8011A
:103DA0000E9495147C01D80115968C91811521F102
:103DB00097013A9521153F4408F055C097013327E4
:103DC000A901445051094432510528F02B523109C0
:103DD0002E30310588F4E091DA04F0E0EE0FFF1F99
:103DE000E855FB4F208131812F3F4FE7340721F009
:103DF0002F5F3F4F31832083909137059111F2C19E
:103E0000811509F4ABC050E4E51652E5F50608F05B
:103E100092C0E11482E5F80680F5E11497E0F90616
:103E200061F138F5C701805E9109089730F1309152
:103E30008E05809191052091860598E0F801A5E214
:103E4000B5E001900D929A95E1F7F0922C05E09281
:103E50002B0510922E05832B822B809324050DC0F9
:103E6000E0E0F0E092CFE114E1E0FE0628F69701F1
:103E7000A7CFE114BFE0FB06D1F6C7019757803802
:103E8000910508F0D1C2BE2CF0E1EF1608F0A0C0F9
:103E90006EE073E080E090E00E94B514811198C05C
:103EA000C12CD12C7601B11026C2E4E02E2EAE0139
:103EB0004F5F5F4F5E834D83AD81BE81E22D1D92CA
:103EC000EA95E9F746015701FFEF8F1A9F0AAF0AFB
:103ED000BF0AC701B6010E94B5148983811509F490
:103EE00077C0813009F088C22601370122E0420EF6
:103EF000511C611C711CC501B4010E94B514382EFF
:103F00008A83811509F464C08FEF830D833008F034
:103F100007C2C301B2010E94B5148B83811519F049
:103F2000CE01019689DA4601570133E0830E911CD8
:103F3000A11CB11C24C2E0EEEE16E2E5FE0638F448
:103F4000F0E6EF16F2E5FF0608F097CF70CF970185
:103F500027573C472530310508F069CF29E7E2169D
:103F60002CE7F20609F046C020912B0530912C0574
:103F7000232B71F1811599F081E00E94F10F80915E
:103F8000240511DB88E0E5E2F5E0ACEDB4E001905A
:103F90000D928A95E1F780912E058093DB0486E0EF
:103FA000F801ACEDB4E001900D928A95E1F78091B3
:103FB000DB04809337058CED94E0BADE1092370570
:103FC000D80115968C91811103C080912405F4DAF3
:103FD000809192058770811549F0F80185818115DE
:103FE00029F08091980582FD0E94C1112996E2E195
:103FF0000C94CB33BAE7EB16BCE7FB0609F0F2C032
:10400000811509F4C7C0A0902B05B0902C05E09154
:104010002405E887E983BE016F5F7F4FC5010E94D9
:104020006D0F2C01F981F987A4EECA2EA4E0DA2ED7
:10403000EE24E394F12C22242A94D60117963C9086
:10404000179733FE54C06D907C90119712968D9007
:104050009C90139746145704B9F41496BC91BF83EF
:10406000232DF60146816B2F89850E94870F8115CC
:1040700059F08F810E944B0C281634F4D601159606
:104080009C917401F92A282E48145904C9F431FE70
:1040900017C0F601F581FF83232DD60116964C91AA
:1040A0006F2F89850E94870F811551F08F810E94A3
:1040B0004B0C28162CF4F60194817301F92A282E52
:1040C00030FE15C0FFEF2F1212C021E0E216F104FE
:1040D00071F4232DD60116964C9160E089850E94DB
:1040E000870F811521F0F60185817401F82AF8E027
:1040F000CF0ED11C24E235E02C153D0509F09DCFF3
:1041000031E0E316F104D9F5988592959F704885C2
:10411000942B9F7081E0403108F480E0F82EF294F7
:10412000F0EFFF22F92AC5019A9581159F4108F504
:10413000FB28BB24EA2C8F2D8D704A2D811509F4A4
:104140004DC06AE080EC99E00E940210282F30E018
:104150002115310551F44E2D66E182EA99E00E9465
:104160000210282F30E0811541F0D901BF297D01CF
:1041700006C0A11481E0B806E8F2E12CF12C86E03B
:10418000EFE2F5E0DF011D928A95E9F7F09236053E
:10419000E09235058091350590913605892B09F41B
:1041A00017CFF8018581811539F08FEF0E94F10F4B
:1041B00080912E0580932D0586E0F801AFE2B5E0F1
:1041C00001900D928A95E1F780912D058093370536
:1041D0008FE295E0ADDD10923705FACE68E088EB0E
:1041E00099E0B2CF811149CEE114A7E5FA0608F4AF
:1041F00036C1E114B8E5FB0608F097C56701E7E5AD
:10420000DE1A68E375E08C2D0E94B315892B31F519
:10421000C60164E0880F991F6A95E1F7FC01EA5B2B
:10422000FA4F2281213009F0EBC0209138053091FE
:104230003905232B99F020913A0530913B05232B2A
:1042400069F020913C0530913D0540913E0550912B
:104250003F05242B352B232B09F4DCC0809142052C
:10426000811143C1C70197558115914008F002C2E1
:1042700057015CEFA522BB24A114B10409F0A8CE1C
:10428000F701FF2754E0EE0FFF1F5A95E1F7CF012A
:104290008A5B9A4F6C01D80115968C91E55BFA4FB9
:1042A000908180FB90F99083811509F4C7C10E9429
:1042B000E11890938A0580938905F60182818F5FCA
:1042C00082838091910590918E05892B83838091C3
:1042D000860584834681578166857785C6010E945D
:1042E0001710D60115968C9181FF5701B092880561
:1042F000A092870526C12FE0C21623E0D206E10472
:10430000F10409F465CEC701B6010E94B5143FEF70
:10431000C31AD30AE30AF30A8111EDCFBA94C3CDCD
:104320008BEF830D833090F54601570143E0840EF7
:10433000911CA11CB11CC301B2010E94B5148B8356
:104340008115E9F0C501B4010E94B5148C83811573
:1043500079F08B819C8181305FEF950710F0982F69
:104360008827A6E03A1671F0B7E03B1669F0E0D571
:104370004601570154E0850E911CA11CB11C75012A
:1043800064019ACD71D5F4CFA1D5F2CFE4E0530109
:1043900042013E12F4CFC301B2010E94B514782E3F
:1043A00046015701F4E08F0E911CA11CB11CC701FE
:1043B000B6016D5F7F4F8F4F9F4F0E94B5147114F0
:1043C00009F406CE811509F403CE8150990B4FEF05
:1043D000489F9001499F300D1124472D4150550BA6
:1043E000240F351F2150310950F28FE99FE00197CA
:1043F000F1F700C00000F6CFCE0101961DD8BFCF67
:10440000223009F02BCF20913C0530913D05232B24
:1044100009F424CFFC01E55BFA4F20812E7F208335
:104420008A5B9A4FFCDB1ACFF3E7EF16FCE7FF0637
:10443000B1F480914205811511F0C8D8C9CD109210
:104440008E050E94350D0E94E11888579C4E90936E
:1044500044058093430581E080934205B9CD22EA6B
:10446000E21622E5F20689F032EBE31632E5F306B6
:1044700049F041EEE416F10441F055EEE516F10481
:1044800009F0ECCE25EE30E002C021EE30E02770DE
:10449000332781E090E001C0880F2A95EAF7209148
:1044A000450530914205311571F0D80115963C91C2
:1044B000311521F0282B209345058ACD8095822344
:1044C0008093450585CD322F3823311509F4CACEA6
:1044D000982F90959223909345050E942D0DF801F9
:1044E0008581811509F474CDBDCEC0908E05D09024
:1044F00086050E94E11888579C4E9093440580934E
:104500004305D80115968C91811509F4ABCE8D2DFC
:104510008C298D7981114FC0B4EBEB16B2E5FB0607
:1045200081F008F051C0F0E4EF16F2E5FF0650F517
:10453000E11422E5F20628F436EEE316F10409F060
:1045400059C0D80115969C91911509F4F5C31092A4
:104550008B05970130572332310508F0FCC384E006
:1045600090E00E94B4349093980580939705F701EA
:10457000E150F047E232F10508F0A9C0E75FFA4CDC
:104580000C944334C7018056924580349105C8F29B
:1045900010929105AEE2EA16F10408F046C0B8E2C6
:1045A000EB16F10488F5EEE1EE16F10488F5C7018B
:1045B00004974A9728F10AD880918E059091450575
:1045C000892B80938E054ECE49E7E4164CE7F4061E
:1045D00058F457E7E5165CE7F50608F0B2CFC701D7
:1045E000805C92458097D3CF8BE7E8168CE7F8067E
:1045F00079F6A7CF109291059DE2E916F10451F6E4
:1046000082E08093910504C0FAE2EF16F10499F676
:1046100080914505811531F08091910592E08927BF
:10462000809391050E9427191DCE2CE4E216F10417
:1046300079F33DE2E31632E0F306E9CFF601448573
:10464000558566857785C6010E941710D601159697
:104650008C9181FF76CFC601C6DA80918705909153
:104660008805E816F90609F06CCF109288051092BB
:10467000870567CFF701E851FC47E730F10508F0FF
:1046800060CFE55DFA4C0C94433426E241EE61EED6
:10469000F801858106C027E245EE65EED801159642
:1046A0008C91EEDA95CC26E241EE60EEF1CF27E276
:1046B00045EE64EEF3CF26E241EE62EEE9CF27E26B
:1046C00045EE66EEEBCF28E241E065EEE1CF80916A
:1046D0009705816080939705609197057091980583
:1046E00084E090E00E94E2340E94EF1A71CC809145
:1046F0009805886080939805EFCF80919705826038
:10470000E9CF809197058460E5CF80919705886017
:10471000E1CF809198058160EDCF8091980582600E
:10472000E9CF809197058061D5CF80919705806210
:10473000D1CF809197058064CDCF0E94EF1A8091F0
:1047400097058068C7CF809197058C60C3CF809113
:1047500098058360CFCF809197058E7FBBCF8091E6
:104760009805877FC7CF809197058D7FB3CF8091C4
:1047700097058B7FAFCF80919705877FABCF8091D7
:1047800098058E7FB7CF809198058D7FB3CF8091AC
:1047900097058F7E9FCF809197058F7D9BCF8091CE
:1047A00097058F7B97CF0E94EF1A809197058F779F
:1047B00091CF80919705837F8DCF809198058C7FD5
:1047C00099CF80919705992782FF939590FB82F965
:1047D00090FB83F97FCF80919805982F909590FB5F
:1047E00080F990FB81F986CF90919705892F8F7B77
:1047F00096FF80646FCF0E94EF1A90919705892FE2
:1048000097FB87F9805866CF61E08EE090E00E94C8
:10481000C83462CF60E0F9CF90919705892F8F7EE1
:1048200094FF806157CF90919705892F8E7F90FFDD
:10483000816050CF90919805892F877F93FF886082
:1048400059CF89E29BC289E283C2F7E7EF16FCE702
:10485000FF0609F128E7E2162CE7F20639F1970185
:10486000205E32452032310530F5911124C03E2DB5
:104870003F7181E090E0AC0102C0440F551F3A95B2
:10488000E2F77A01642F83E090E00E94C8348E2D15
:104890000E94610C9DCB81E0911551F00E94670C44
:1048A00043E062E081E00E940E0D92CB82E0F4CF03
:1048B0000E94710CF5CF40918D0580919005282FB5
:1048C00030E02095309570E024233723232B19F016
:1048D000482340938D055BE7E5165CE7F50641F458
:1048E000911509F475CB0E944E0C0E94CA0F70CB33
:1048F00080E4E81682E5F80608F077C0A0E2EA1640
:10490000A2E5FA0608F078C097013055211532402B
:1049100008F488C09115C9F0EAE5EE16ECE7FE064A
:1049200009F4C6C008F09BC021E0E2162CE7F206AD
:1049300009F4BCC033E0E3163CE7F30609F4B0C069
:10494000E1144CE7F40609F49EC0D80116968D9147
:104950009C91009709F4B0C00E94330E7C01D801ED
:104960001596DC908091920587708115B9F0BD2C69
:10497000D114A9F08F2D807F803421F080E28E0D3C
:10498000883060F08091980582FF08C00E94C111B4
:10499000809192058770BB24B3948111B12C8F2D27
:1049A00082958F70883009F40AC108F09DC082306A
:1049B00008F4ADC0843009F4E7C0B11409F42FC184
:1049C0008091920580FD2BC1F80115828695869510
:1049D00086950E94670CC801ABD980919205869597
:1049E000869586950E94710C1AC19701205C32450C
:1049F0002032310508F08ECF8E2D8F7120918D05DC
:104A000030E041E050E0082E02C0440F551F0A94E8
:104A1000E2F724233523232B09F47CCF911509F4E5
:104A2000D7CA63CF970145E0369527954A95E1F7B8
:104A3000822F8F7020918D0530E041E050E0082EEC
:104A400002C0440F551F0A94E2F724233523232B79
:104A500009F460CF911149CF10928E0591C15BE5A9
:104A6000E5165CE7F50631F18CE5E8168CE7F8060B
:104A700009F06BCF80919805002482FF0394802D6C
:104A80000E94781362CF0E94EF1A9FEFA4E3BCE06C
:104A90009150A040B040E1F700C000000E94F21227
:104AA0006FEF7FEF80E090E00E94E2340E940F1BE6
:104AB00081E0E6CF80E0E4CFF8018581C080D1803D
:104AC000811569F0C6010E946C14F82E682FC6018A
:104AD0000E94D50CB6018F2D0E9442143DCFC60115
:104AE0000E94F20CF82EF6CF893009F4DDC08A5FFF
:104AF0008F70823008F061CFB2EFEB12E8C08F2DDB
:104B00008F71D11409F4EEC00E94710C56CFEF2DB5
:104B1000EF70CE2EF0E1FF1618F0C29480EFC8229D
:104B2000D114C9F0C11469F080E28E0D883010F004
:104B3000E1100BC080918E058C2980938E050E9418
:104B400027198E2D0E947B1938CF809191058C29D1
:104B500080939105F4CF8E2D0E94DF19C11409F4C2
:104B60002CCF80E28E0D883010F0E11006C08C2D25
:104B70000E942D0D0E94271920CFC094809191058D
:104B80008C2180939105F6CF8F2D86958695837025
:104B9000811561F0813009F010CFC7019370D110F9
:104BA00002C080E090E00E94531007CFC7019370CD
:104BB000D11002C080E090E00E942B10FECE8F2D1D
:104BC0008370811139C0D11028C04E2D4295469571
:104BD0004770440F440F8E2D8F70042E01C0880F34
:104BE0000A94EAF72E2D2071E4FE07C02FE030E092
:104BF00001C0220F4A95EAF720953F2D369536954C
:104C000033703230A1F0333081F040918F05313074
:104C100059F0822B84230E94610C0E941C1060E0DA
:104C2000C8010E949514E2C9842B822BF4CF822BF9
:104C300090918F058927EFCFD11459F1F0FEEDCF78
:104C40004E2D429546954770440F440F8E2D8F7020
:104C5000042E01C0880F0A94EAF72E2D2071E4FE7D
:104C600007C02FE030E001C0220F4A95EAF72095F7
:104C70003F2D369536953370323089F0333069F0F8
:104C800040919005313041F0822B84230E94640CC6
:104C9000C4CF823010F2D4CF842B822BF7CF822B5B
:104CA000909190058927F2CF2F2D2F70F22ED114DD
:104CB00039F0822F0E94670C8E2D0E94C41AADCF4E
:104CC0008E2D0E94CD1A8F2D0E94710CA6CF33EF2E
:104CD000E31659F041EFE41216C08F2D8F71D114F5
:104CE00009F412CF0E94670C68CE80E0D11441F025
:104CF0005F2D5F71F52E81E001C0880F5A95EAF7AC
:104D00000E94640C5ACED1101CCF89E3E81209C06E
:104D10009FEFA7EEB3E09150A040B040E1F700C094
:104D200000008E2D0E94DF1948CEB3E7EB16BCE7DA
:104D3000FB0609F44DC992CAE6E1EE16ECE7FE0661
:104D400009F083CD80918C05811509F47CCD85E334
:104D50000E94AF1015C0F6E1EF16FCE7FF0609F060
:104D600074CD80918E058A7A91E0811101C090E026
:104D700090938C05811509F464CD85E30E947B1026
:104D80000E94271925C9AEE0B0E0E9ECF6E20C94E8
:104D9000BD3349875A876B877C878D879E879111A2
:104DA0001092910518861F8226E0FE013996CE01E9
:104DB0000196DC0101900D922A95E1F7209198056A
:104DC0008C0122FF1DC00E94E118209193053091B3
:104DD0009405821B930B8838934128F080919205AB
:104DE00082FF0E94C1110E94E11820919505309127
:104DF0009605821B930B8838934110F00E94350D65
:104E00008D81811541F061E0C8010E94951461E037
:104E1000C8010E949514C8010E94981E2E96E4E0D5
:104E20000C94D933A6E0B0E0E8E1F7E20C94BD338E
:104E30000E94E1188C018091730490917404801792
:104E4000910771F019821A820E94E118BC01498110
:104E50005A8180E090E097DF10937404009373040C
:104E60002696E4E00C94D933A6E0B0E0EAE3F7E25A
:104E70000C94BD338C019093700480936F040115E2
:104E800080E21807B0F4C801805E9109089728F005
:104E900063ED7AE10115110511F464EC7AE1C801C2
:104EA0000E941F0C802F0E947B192696E4E00C9430
:104EB000D93380EF89838A830E94E1188160BC0125
:104EC00049815A8181E091E05EDFEFCFA6E0B0E05A
:104ED000ECE6F7E20C94BD338C0190937004809360
:104EE0006F04011580E21807B0F4802F0E94DF19CB
:104EF000C801805E9109089728F06CED7AE10115F0
:104F0000110511F46DEC7AE1C8010E941F0C269680
:104F1000E4E00C94D93380EF89838A830E94E118FE
:104F20008160BC0149815A8181E090E02CDFEFCFA4
:104F3000CF93DF93D82FC92F97DF8D2F9C2FC6DFFC
:104F4000DF91CF9108950F931F93CF93DF938C013F
:104F5000862F68E375E00E94B315892B91F4C09108
:104F60003805D0913905209761F0F80182818330AE
:104F700039F4CE01DDDFCE01DBDFCE01D9DF01C0A8
:104F8000E0F7DF91CF911F910F9108950F931F9339
:104F9000CF93DF938C01EB0168E375E08C2F0E94C7
:104FA000B315892B09F057C0FE01FF27D8011296CF
:104FB0008C911297EF5CFD4F8130A9F415968C917E
:104FC00082FD4EC080FF4CC082E0808380913A0514
:104FD00090913B050097B9F480913805909139057F
:104FE0000097C9F110C08230A1F515968C9182FD11
:104FF00026C080FD0AC083E0808380913C059091AB
:105000003D050097F1F030DF26C084E08083809179
:105010003E0590913F050097B1F78091380590913A
:105020003905009701F184DF80913A0590913B05A5
:10503000009749F78091380590913905E4CF85E0D4
:1050400080838091380590913905009721F070DFB9
:10505000F1CF86E08083DF91CF911F910F9108956A
:1050600081E08083B9CF80913A0590913B05B8CF1C
:105070000F931F93CF93DF938C01EB0168E375E0EF
:105080008C2F0E94B315892B71F4DD27CF5CDD4F87
:105090008881F801128218828330E9F048F4813067
:1050A00059F0823081F0DF91CF911F910F910895D7
:1050B0008430B1F08530B9F7809138059091390589
:1050C000009789F306C080913A0590913B050097BF
:1050D00099F3FCDEE8CF80913C0590913D05F7CF38
:1050E00080913E0590913F05009799F720913805F2
:1050F0003091390580913A0590913B052115310594
:10510000F9F2009731F7C901E4CFA4E0B0E0EBE891
:10511000F8E20C94B233FE01319684E0DF011D9277
:105120008A95E9F789E3E82E81E0F82E8F019DE367
:10513000C92E91E0D92E3F01AA24A394B12C30E4CA
:10514000832E31E0932EF70181917F018F3F09F487
:105150003EC0F894E82FE295EF70F0E021A18F7047
:10516000A50102C0440F551F8A95E2F7CA01922F8C
:10517000982B91A392A18095892382A3789400C053
:10518000EDE3F1E031E0512C21912F3F79F0A22F96
:10519000A295AF70A05EB0E08C9190E02F7002C03D
:1051A000959587952A95E2F780FF39C080E0582AC7
:1051B000330F8E169F0641F7F70182918F3F11F052
:1051C0000E942F0F50EA5A95F1F7D8015C920F5FB9
:1051D0001F4FCE14DF0409F0B6CF44E050E0B30116
:1051E00085E392E00E948834892BD9F089819A81E5
:1051F000AB81BC818093350290933602A093370235
:10520000B093380281E08093E8010E94E118909306
:10521000E7018093E6012496EFE00C94CE33832FD0
:10522000C6CF8091E8018115B1F30091E60110919C
:10523000E7010E94E118801B910B059760F344E0A1
:1052400050E065E372E088E694E00E948834892BA0
:1052500081F08091350290913602A0913702B09191
:1052600038028093680490936904A0936A04B09311
:105270006B041092E801CFCFCDB7DEB7E8970FB639
:10528000F894DEBF0FBECDBF85B7806885BF85B7F8
:10529000806885BF84B7877F84BF0FB6F894A895D0
:1052A00080916000886180936000109260000FBE62
:1052B00080E890E00FB6F8948093610090936100CD
:1052C0000FBE81E0809318018DE29FE09093BD01B5
:1052D0008093BC010E94550F0E9477150E94941183
:1052E0000E9498128091E20084608093E20078949A
:1052F00080916E04811599F08091E9001091EC0085
:105300008F70179511271795182B1092E90080912F
:10531000E80083FD0E94241B1F701093E90082E0C7
:1053200084BD93E095BD9AEF97BD80936E000E9477
:10533000C614811102C00E944216EAE5F4E088E03A
:10534000DF011D928A95E9F781E08093590460E0BE
:1053500080E00E94A80F61E080E00E94A80FEFE8C3
:10536000F1E03197F1F700C0000010E0809159049E
:10537000181708F47CC087EF0E942F0F87E90E945E
:105380002F0F86E60E942F0F84E90E942F0F84EFD3
:105390000E942F0F85EF0E942F0F86EF0E942F0F84
:1053A00084E0E8E6F4E0DF01282F1D922A95E9F772
:1053B000E5E3F2E0DF011D928A95E9F780E090E0F5
:1053C0000E94B434833E9E4F21F40E94C614811182
:1053D00029C063EE7EEF80E090E00E94E23460E05E
:1053E00082E090E00E94C83481E080938F0561E004
:1053F00083E090E00E94C83460E074E184E090E0D3
:105400000E94E2340E94421640E050E0BA018FE070
:1054100090E00E94DA3440E050E0BA0183E190E08D
:105420000E94DA3482E090E00E94AC348093480419
:1054300084E090E00E94B43490939805809397059F
:1054400064DEEFEFF6E721E0E150F0402040E1F7C5
:1054500000C000005ADE8091690480FF1AC06FEF1F
:105460007FEF80E090E00E94E2340E94F21260E060
:10547000812F0E94BC0F082F61E0812F0E94BC0F7A
:10548000E12FF0E0E85AFB4F880F802B80831F5FED
:105490006DCF83E090E00E94AC340E94610C82E00A
:1054A0008093450480E8809344040E9485326BE039
:1054B00070E08BEA98E00E94C815811509F43FC09E
:1054C0008091450465E070E081FD8FC086EA98E038
:1054D0000E94C815811599F16DE070E084E998E0AB
:1054E0000E94C815811559F10E94DE10DC01CB0124
:1054F000805A9541AF4FBF4F809340049093410431
:10550000A0934204B0934304EDE3F2E080E092E024
:10551000DF019C011D9221503040E1F7F0933C02E5
:10552000E0933B028FEF9FEF90933A028093390212
:1055300081E080933F0480933E0410923D0488E014
:1055400091E0909396048093950480916E0410E40A
:1055500000E1F2E1FF2E853009F47EC0D6DD09E4DA
:1055600014E0E8E6EE2EE4E0FE2ED701F80191917A
:105570008D9124E0ED34F20709F478C09817B9F35F
:10558000D12CD701CD907D01F80191908F019C1411
:1055900021F19C24B12CAA24A394892D8A21811560
:1055A000A9F0B982DA820E94E1189C838B83F1E032
:1055B000FD8391E08C2D8A21811101C090E09E83B2
:1055C00049815A816B817C818D81DDDBB394AA0C8A
:1055D00023E0B212E2CFF801C292D39434E0D312A6
:1055E000D0CF0E94DE1001E045C081EA98E070CF84
:1055F00080916E04843029F10E94D51510924604E2
:1056000048E150E00FB6F894A895409360000FBEB3
:105610001093600083B7817F846083BF83B781600C
:1056200083BF7894889583B78E7F83BF0FB6F89435
:10563000A89580916000886180936000109260005E
:105640000FBE63DDE8E6F4E08191811198C58CE638
:1056500094E08E179F07C1F780916E04853009F49E
:10566000C7CF0E94EF1A0E941C1078CF981388CFE2
:10567000D9DB00E0E0908705F0908805E114F104A3
:1056800001F1C0908905D0908A050E94E1188C191B
:105690009D09893C9105A8F0C70199274CEFE422A8
:1056A000FF24EF2809F0E9C074E0880F991F7A956C
:1056B000E1F78A5B9A4FDC0115962C9122FF0E943C
:1056C0000F1E8090A8049090A904092C000CAA0831
:1056D000BB0810911401212F30E0E8EAF4E081E0EA
:1056E00090E03296281739070CF0CAC0C0905304D6
:1056F000D0905404E0905504F09056040E94DE10BF
:105700002B013C014C185D086E087F089401A5012F
:10571000B7FE04C020E030E040E050E0A0E6BAEE82
:105720000E9460346B017C01B8EC1B9F9001112436
:10573000032E000C440B550B240D351D461D571D23
:10574000A5E0B0E00E9460349B01AC01C701B60146
:105750000E94053469017A01213F31054105510557
:1057600010F060EFC62EF9EC4F165104610471047D
:105770000CF18091DA0490E0019669E170E00E94FA
:10578000F2338093DA04880F991FFC01E855FB4F30
:1057900011821082183108F017E11F5F1093140175
:1057A0000E94DE1060935304709354048093550458
:1057B0009093560422E082169104A104B1040CF4E3
:1057C000C12C80904F0490905004A0905104B09050
:1057D00052040E94DE109B01AC01281939094A09C4
:1057E0005B0949015A0135E683169104A104B1040D
:1057F00084F00E94DE1060934F04709350048093F5
:105800005104909352048091990580934E04C09264
:105810004D0410914E04A0914D04A11BBB0BA5019A
:1058200094010E946A3424E630E040E050E00E9497
:105830002734120F1093990580914205811569F064
:105840000E94E1182091430530914405821B930B7F
:105850008F3F9F4710F40E94E61A809162048115E1
:1058600051F080915C041092620480935D048091F9
:105870005A0480935B04F12C58C080E090E01BCF69
:1058800040815181052E000C660B770B840E951E0E
:10589000A61EB71E019625CF61E08F2D0E94BC0F7A
:1058A000E82E60E08F2D0E94BC0FEE0CE82A2F2D11
:1058B00030E0D901A85ABB4FEC918E2F8370E816C7
:1058C00099F1EE0FEE0FEE29EC93EF70F0E0E05C53
:1058D000FE4F295A3B4F8081D9019C91890F8C93AF
:1058E00084300CF453C0412F50E0BA016F5F7F4FFA
:1058F00063707727D616170679F0465A5B4F9F2DAF
:105900009F77FA0194831F5F137010935C0490914A
:105910005A049F5F90935A04082E000C990B64E080
:1059200070E060D7F9018083F394D0905D0410910A
:105930005C0480915904F81608F4AECF90E03CEF77
:10594000E32E4DEFD42E80915D0420915C04281746
:1059500009F455C0E82FF0E0E25AFB4F908197FB25
:10596000CC24C0F8F92EE894F7F88F5F8370809309
:105970005D0480915B048F5F80935B0497FD1BC087
:10598000FBA6ECA60E94E11813E01AC08D3F24F696
:10599000412F50E0BA016F5F7F4F63707727D616B3
:1059A000170609F4B9CF465A5B4F9F2D9068DA016C
:1059B00014969C93A8CFFBA6DCA60E94E11812E0E7
:1059C000BC018DA79EA71FA7F1E0F8AB4BA55CA576
:1059D000812F91E0D8D9F9AAC11479F0DAAA0E94EE
:1059E000E118BC018BAB9CAB1DAB1EAA49A95AA9FF
:1059F000812F90E0C8D991E0A6CFEAAAF0CF911507
:105A000039F00E94DE100E9411170E94E61504C0B2
:105A10000E9411170111F9CF0E941C10909163048C
:105A2000891721F0809363040E94DE1080916E0438
:105A3000843009F08ACD83E08093E9008091E8000A
:105A400082FF83CD8091E80090E085FF05C00E9431
:105A50006311811519F191E08091E8008B778093B3
:105A6000E800911509F471CD009171041091720450
:105A7000E9810115110579F1EE3F09F04EC08A81E7
:105A8000833020F08550833008F047C0EA81EE3043
:105A900008F043C0F0E0EE5CFA4CF5C600E210E01E
:105AA0009E012F5F3F4F79018091E80085FD0AC07C
:105AB0008091E8008B778093E8000E946311811544
:105AC00099F3C9CF8091F100D7018D937D010150E9
:105AD000104051F7C0CFE43148F4E11549F0E150EE
:105AE000E33130F4F0E0E05CFA4CCDC6EE3F71F209
:105AF0008FEF898312C01A8289E08B830EC08A815E
:105B0000823081F08330B1F0813091F70E94DE1055
:105B1000D0D66B837C838D839E83CE0101960E94B9
:105B2000B31113CD88E290E017D71B821C821D822F
:105B30008E83F3CF80916C0490916D04892B69F36F
:105B4000809168048B83809169048C8380916A04BE
:105B50008D8380916B04ECCF8A81823049F66B8112
:105B60007C818D819E81A5D688E290E011D7D5CF2A
:105B70004C816B818A810E94E0139827892798279E
:105B80009E838D83CACF2D813E81322723273227E2
:105B90004C816B818A810E948D13BFCF0E94DF14DC
:105BA000BCCF80E18A83B9CF83E08A838FE0A5CF21
:105BB0008C818D3108F0B1CF8A809B809824892414
:105BC0009824A12CB12C8E010F5F1F4F7801E80E95
:105BD000F11CE016F10609F4A0CF80E0BFE08B16BF
:105BE000B3E09B06A104B10420F4C4018F509F4F81
:105BF000B3D6F80184830F5F1F4FFFEF8F1A9F0A00
:105C0000AF0ABF0AE6CF80916C0490916D04892B96
:105C100009F483CF8C818D3108F07FCF882E912CB1
:105C2000A12CB12CCA80DB80DC24CD24DC24E12C27
:105C3000F12C8E010F5F1F4F412C512C3201481463
:105C400059046A047B0408F068CF2FE0C21623E0F1
:105C5000D206E104F10438F4D80114966C91C6011F
:105C60008F509F4F95D6BFEF4B1A5B0A6B0A7B0A8A
:105C7000EFEFCE1ADE0AEE0AFE0A0F5F1F4FDFCFEC
:105C80000E9408164ACF84E08DCF8C818D3108F0B8
:105C900044CF882E912CA12CB12CCA80DB80DC242F
:105CA000CD24DC24E12CF12C412C512C32018E012D
:105CB0000B5F1F4F481459046A047B0408F02DCF72
:105CC00080E0F0E6CF16D104E104F10418F4C60137
:105CD000899642D6D8018D938D01BFEF4B1A5B0A8E
:105CE0006B0A7B0AEFEFCE1ADE0AEE0AFE0AE2CF5B
:105CF0002C81022F10E02D3108F00FCF8A819B817B
:105D00009827892798272C01612C712C80369105C2
:105D100008F003CF822E912CA12CB12C40E650E04C
:105D200060E070E04419550966097709421751058A
:105D30006105710508F4F1CE20916C0430916D0479
:105D4000232B09F03FC01C01F9E22F0E311C80FB10
:105D5000EE24FF24E0F880FF0BC08896FDD59D81DE
:105D600089279827892781159C4711F48FEF8D8308
:105D7000D501C401840D951DA61DB71D80FF1AC055
:105D8000680131E0C31AD108AE014B5F5F4F4C0D83
:105D90005D1D58AF4FABC101800F911FDDD5AFA97D
:105DA000B8AD9C9181159C4721F48FEFEFA9F8AD18
:105DB00080838601FE013196EE0DFF1D2FEFE01668
:105DC000F10638F08E010F5F1F4FC12CD12C7601E8
:105DD00024C09481858181159C4711F424832583F7
:105DE00042E0E40EF11C3296EACF50E6451651042B
:105DF0006104710430F4D80114966C91C201899643
:105E0000C7D5BFEFCB1ADB0AEB0AFB0AEFEF4E1A3E
:105E10005E0A6E0A7E0A0F5F1F4FC814D904EA0497
:105E2000FB0418F37ACE80916C0490916D04892B59
:105E300009F473CECE0101960E94B311FFEF21EE5B
:105E400034E0F15020403040E1F700C000000DCBBD
:105E500088E0E9E1F1E0DE01919601900D928A95EA
:105E6000E1F7FE0132968FE1DF011D928A95E9F795
:105E700086E0898388E07F96DE01159601900D9279
:105E80008A95E1F74ACE8CEE89831A821B821C82A6
:105E900044CE8B819C81092E000CAA0BBB0B25E004
:105EA000880F991FAA1FBB1F2A95D1F7AC01BD010E
:105EB000405E5F4F6F4F7F4F481759076A077B0758
:105EC00008F42BCE8C3E9105A105B10508F025CE36
:105ED0004D3E51056105710520F04CEE50E060E04B
:105EE00070E0481B590BBC016A54774FCE010196F4
:105EF00006D513CE1B810C8140E0602F812F0E94BC
:105F00000F149827892798279A83898341E0602F67
:105F1000812F0E940F149827892798279C838B83B1
:105F2000FCCD8E819F819827892798270E94480F52
:105F30009C0141E08D81811101C040E06C818B8129
:105F40000E94B413EACD4AE150E06FEF70E0CE0159
:105F50000796EBD480916C0489830A831B821C8290
:105F60001D8282E0E5CD81E090E090937204809301
:105F7000710482E390E090936704809366040E942A
:105F8000E1189093650480936404C7CD0115110551
:105F900071F1D0906804E0906404F09065040E9470
:105FA000E1188E199F098536910540F1D2FE26C071
:105FB000D0FE24C00E94E11890936504809364048D
:105FC0008091660490916704019790936704809391
:105FD0006604892B61F4109272041092710481E0BE
:105FE00090E090936D0480936C0400E010E0809149
:105FF0006C0489830A83809166047FCD82E390E0FC
:106000009093670480936604F2CF10926D0410920F
:106010006C0483CD40E250E06FEF70E0CE0101965A
:1060200084D47BCD8B81823009F457C080F48111F8
:106030003DC0FE0132968EE1DF011D928A95E9F79F
:1060400084E0898388E08C8383E088A366CD8730F1
:1060500009F478C0883009F060CD1C8186E0FE012B
:106060003596DE01919601900D928A95E1F789A10E
:106070009AA10E94480F9AA389A38BA19CA10E9478
:10608000480F9CA38BA38FEF183060F4F6E01F9F9E
:10609000B00111246F537F4F46E050E0CE0181964E
:1060A00095D480E089830E94771537CD8C819AE062
:1060B000F92E8E010F5D1F4FF8012F2D11922A9599
:1060C000E9F7B8010E94B3158983F801DE01129641
:1060D00001900D92FA94E1F720CD1C818AE0FE0137
:1060E0003596DE01919601900D928A95E1F789A18E
:1060F0009AA10E94480F9AA389A38BA19CA10E94F8
:10610000480F9CA38BA38DA19EA10E94480F9EA324
:106110008DA38FA198A50E94480F98A78FA38FEFFA
:10612000143060F43AE0139FB001112467567F4F9A
:106130004AE050E0CE01819649D480E089830E94F4
:10614000550FEBCC2C8166E0CE018196DC01E62F69
:106150001D92EA95E9F7283080F4629FB00111247E
:106160006F537F4F46E050E0E7D380E0898386E0BD
:10617000FE01B196DE01129681CE8FEFF7CF8091AE
:106180004704811509F468CA09BDF9BC09B400FEC9
:10619000FDCF8091D8008F7D8093D8008091E00062
:1061A00082608093E0008091E00081FDFCCF0E943E
:1061B000EF1A52CA78941F921FB61F9211248F9320
:1061C0009F93AF93BF938091040290910502A09199
:1061D0000602B09107020196A11DB11D8093040231
:1061E00090930502A0930602B0930702BF91AF916E
:1061F0009F918F911F901FBE1F9018951F920F9215
:106200000FB60F9211242F933F934F935F936F9389
:106210007F938F939F93AF93BF93EF93FF9380915F
:10622000E10082FF09C08091E20082FF05C08091F9
:10623000E1008B7F8093E1008091DA0080FF24C031
:106240008091D80080FF20C08091DA008E7F8093FB
:10625000DA008091D90080FFA9C080E189BD82E188
:1062600089BD09B400FEFDCF81E080936E0480916A
:10627000F301811109C00E9494110E94981280912B
:10628000E20084608093E2008091E10080FF1AC008
:106290008091E20080FF16C08091E2008E7F8093A3
:1062A000E2008091E20080618093E2008091D8005A
:1062B00080628093D80019BC85E080936E0483E0EF
:1062C000809318018091E10084FF2FC08091E2004B
:1062D00084FF2BC080E189BD82E189BD09B400FE45
:1062E000FDCF8091D8008F7D8093D8008091E10010
:1062F0008F7E8093E1008091E2008F7E8093E200A8
:106300008091E20081608093E2008091F20181152A
:1063100009F452C084E080936E0480916E0484304E
:1063200009F052C082E0809318018091E10083FF60
:106330002CC08091E20083FF28C08091E100877F1C
:106340008093E10082E080936E041092F2018091CC
:10635000E1008E7F8093E1008091E2008E7F809348
:10636000E2008091E20080618093E20042E060E020
:1063700080E00E9468128091F00088608093F000B5
:1063800081E08093180180931701FF91EF91BF91F5
:10639000AF919F918F917F916F915F914F913F91BD
:1063A0002F910F900FBE0F901F90189519BC10924F
:1063B0006E041092F30168CF8091E30087FF02C062
:1063C00083E0A9CF81E0A7CF81E0ADCF1F920F92EC
:1063D0000FB60F921124EF92FF920F931F932F93FA
:1063E0003F934F935F936F937F938F939F93AF935D
:1063F000BF93CF93EF93FF9309EE10E0F8018081F4
:10640000C091EC008F70C795CC27C795C82B108220
:1064100080EFE82EF12CF7018081877F80837894CC
:106420000E94241BF8011082F7018081886080831C
:10643000CF70F801C083FF91EF91CF91BF91AF91E1
:106440009F918F917F916F915F914F913F912F918C
:106450001F910F91FF90EF900F900FBE0F901F9024
:106460001895FF920F931F93CF93DF93182FEB0193
:106470001092BC0084EA8093BC000E94E118082FAF
:10648000F92E8091BC0087FF28C08091B900887FD9
:10649000883029F08091B900887F803199F5109378
:1064A000BB0084E88093BC000E94E118182F092FDC
:1064B0008091BC0087FF1EC02091B900287F80E03A
:1064C00090E0283199F081E090E0203411F480E0F0
:1064D00090E091958195910909C0802F9F2D0E9490
:1064E000371EC817D90768F68EEF9FEFCDB7DEB716
:1064F000E5E05EC1812F902F0E94371EC817D90793
:10650000B8F6F2CF8FEF9FEFF1CF1092B9008CE089
:106510008093B80008950F931F93CF93DF93EB01FF
:106520008093BB0084E88093BC000E94E118182F80
:10653000092F8091BC0087FF11C02091B900287FEE
:1065400081E090E0283211F480E090E0919581950F
:106550009109DF91CF911F910F910895CF3FDC07F3
:1065600041F3812F902F0E94371EC817D90708F7D3
:106570008EEF9FEFEECFA0E0B0E0E0ECF2E3F4C0EE
:10658000782EB62EA72E6A0189010E94E1184C01CF
:106590000431110508F10F3F100711F1C80164E142
:1065A00070E0C9D0F62EE72E6F2D7E2D872D59DF96
:1065B000EC01892BC1F4EB2CFA2CCE0CDF1CEC1473
:1065C000FD0411F02097C9F084E98093BC00CE014E
:1065D000CDB7DEB7EDE0E4C0FF24F394E12CE4CFC7
:1065E00085E0F82EFBCF0F3F1007F1F2C4010E94A7
:1065F000371E08171907C0F6DECFB801F7018191E1
:106600007F0189DFEC01DBCFA0E0B0E0E9E0F3E35C
:10661000ABC0782EB62EA72E6A0189010E94E11820
:106620004C010431110508F10F3F100711F1C801A9
:1066300064E170E080D0F62EE72E6F2D7E2D872D41
:1066400010DFEC01892BC1F4EB2CFA2CCE0CDF1CF3
:10665000EC14FD0411F02097C9F084E98093BC008C
:10666000CE01CDB7DEB7EDE09BC0FF24F394E12C63
:10667000E4CF85E0F82EFBCF0F3F1007F1F2C40105
:106680000E94371E08171907C0F6DECFF701849164
:10669000B80141DFEC01FFEFEF1AFF0AD9CFA0E00C
:1066A000B0E0E4E5F3E35FC0682E962E5A0169017D
:1066B00078010E94E118782E892E0431110518F115
:1066C0000F3F100719F1C80164E170E034D0162FB4
:1066D000072F612F702F862DC4DEEC01892BC1F0AE
:1066E000FFEFEF16FF06A9F3872D982D0E94371EA6
:1066F000E816F90670F784E98093BC00CE01CDB7A7
:10670000DEB7EEE04CC011E000E0E3CF15E0FCCFD7
:10671000B701892D00DFEC018501CA0CDB1C0C15CB
:106720001D0549F3209739F7B701F80181918F01D1
:10673000F2DEEC01F4CFAA1BBB1B51E107C0AA1F7C
:10674000BB1FA617B70710F0A61BB70B881F991F12
:106750005A95A9F780959095BC01CD0108952F9287
:106760003F924F925F926F927F928F929F92AF92E1
:10677000BF92CF92DF92EF92FF920F931F93CF932E
:10678000DF93CDB7DEB7CA1BDB0B0FB6F894DEBFC5
:106790000FBECDBF09942A88398848885F846E84EB
:1067A0007D848C849B84AA84B984C884DF80EE8035
:1067B000FD800C811B81AA81B981CE0FD11D0FB63E
:1067C000F894DEBF0FBECDBFED010895992778E0A4
:1067D000880F991F961708F0961B881F7A95C9F79E
:1067E0008095089597FB072E16F4009406D077FD48
:1067F00008D0A1DF07FC05D03EF4909581959F4F0E
:106800000895709561957F4F0895A1E21A2EAA1BF5
:10681000BB1BFD010DC0AA1FBB1FEE1FFF1FA21750
:10682000B307E407F50720F0A21BB30BE40BF50B4D
:10683000661F771F881F991F1A9469F760957095D6
:10684000809590959B01AC01BD01CF010895052E67
:1068500097FB16F400940FD057FD05D0D6DF07FC48
:1068600002D046F408C050954095309521953F4F91
:106870004F4F5F4F089590958095709561957F4F2C
:106880008F4F9F4F0895EE0FFF1F0590F491E02D5D
:106890000994082E817006940694811D0694811D2A
:1068A0000694811D0694811D0694811D0694801D09
:1068B00008956927962769277827872778270895D5
:1068C0000FD0A59F900DB49F900DA49F800D911D9A
:1068D00011240895B7FFF4CFF3DF821B930B0895C3
:1068E000A29FB001B39FC001A39F700D811D112411
:1068F000911DB29F700D811D1124911D0895FB0102
:10690000DC0102C005900D9241505040D8F7089527
:10691000FB01DC0104C08D910190801921F44150EC
:106920005040C8F7881B990B0895DC0101C06D9396
:1069300041505040E0F70895DC01CB01FC01F9998A
:10694000FECF06C0F2BDE1BDF89A319600B40D92BB
:1069500041505040B8F70895F999FECF92BD81BDDE
:10696000F89A992780B50895A8E1B0E042E050E098
:10697000E5CFDC01A40FB51F4150504040F0CB01E2
:10698000840F951F2E9105D041505040D8F708959F
:10699000262FF999FECF92BD81BDF89A019700B4D8
:1069A000021639F01FBA20BD0FB6F894FA9AF99A78
:1069B0000FBE08950396272FECDFEADF252FE9DFCE
:1069C000242FE7CF0196272FE4DFE2CFDC01CB01B4
:1069D00002C02D9105D041505040D8F70895262F80
:1069E000F999FECF1FBA92BD81BD20BD0FB6F894B4
:1069F000FA9AF99A0FBE01960895F894FFCF051CF4
:106A00002B1C311C2B1C311C841CA61C311CAD1DE5
:106A1000BA1DAB231324B3237D238123B7238523FE
:106A2000BB23C72391230C249523CB239923CF2366
:106A3000F4239D23D323FB23A323D923E1238923F9
:106A4000BF238D23C323A723DD23EB2304240A24A0
:106A50007723AF231A245323572345234B235B2348
:106A60005F236323282F432F492F7A2F912FA32FA2
:106A7000B32FC62F05300A308D2D8D2D8D2D123060
:106A80007B2D7F2DAC2DB82DC32DCE2D782D782DBF
:106A9000782D782D132FD12DD42DD82D032E402EC7
:066AA000432E452E782E66
:106AA600FF0021007F220003DB1058136E13EA104B
:106AB60073134F13010000010008DB6F2840FD6FC0
:106AC600580044226D3B011901AC0085079E07BEA4
:106AD600070008101818100800F7976694F4F5F6E2
:106AE60000FF0100010000FFFF0000010001FF00A0
:106AF600E200E900EA00B500B600B700CD00830168
:106B0600CC008A019201940121022302240225026B
:106B1600260227022A02B300B4006F0070009F010C
:106B2600CB019F02A002E200E900EA00B500B60030
:106B3600B700CD008301CC008A01920194012102A5
:106B4600230224022502260227022A02B300B400E9
:0C6B56006F0070009F01CB019F02A002A5
:00000001FF
